 browser_support

 Timestamp is 5c7621cd (Wed Feb 27 12:36:13 2019)

 Preferred load address is 10000000

 Start         Length     Name                   Class
 0001:00000000 0000050bH .text$di                CODE
 0001:00000510 000030eeH .text$mn                CODE
 0001:00003600 0000054aH .text$x                 CODE
 0001:00003b50 0000012bH .text$yd                CODE
 0002:00000000 00000238H .idata$5                DATA
 0002:00000238 00000004H .CRT$XCA                DATA
 0002:0000023c 00000038H .CRT$XCU                DATA
 0002:00000274 00000004H .CRT$XCZ                DATA
 0002:00000278 00000004H .CRT$XIA                DATA
 0002:0000027c 00000004H .CRT$XIAA               DATA
 0002:00000280 00000004H .CRT$XIC                DATA
 0002:00000284 00000004H .CRT$XIZ                DATA
 0002:00000290 00000478H .rdata                  DATA
 0002:00000708 00000078H .rdata$debug            DATA
 0002:00000780 000002c0H .rdata$r                DATA
 0002:00000a40 00000048H .rdata$sxdata           DATA
 0002:00000a88 00000004H .rtc$IAA                DATA
 0002:00000a8c 00000004H .rtc$IZZ                DATA
 0002:00000a90 00000004H .rtc$TAA                DATA
 0002:00000a94 00000004H .rtc$TZZ                DATA
 0002:00000a98 00000714H .xdata$x                DATA
 0002:000011b0 00000058H .edata                  DATA
 0002:00001208 0000008cH .idata$2                DATA
 0002:00001294 00000014H .idata$3                DATA
 0002:000012a8 00000238H .idata$4                DATA
 0002:000014e0 00001498H .idata$6                DATA
 0003:00000000 00000034H .data                   DATA
 0003:00000034 00000168H .data$r                 DATA
 0003:000001a0 0000041cH .bss                    DATA
 0004:00000000 00000058H .rsrc$01                DATA
 0004:00000060 00000180H .rsrc$02                DATA

  Address         Publics by Value              Rva+Base       Lib:Object

 0000:00000000       ___guard_flags             00000000     <absolute>
 0000:00000000       ___guard_fids_table        00000000     <absolute>
 0000:00000000       __except_list              00000000     <absolute>
 0000:00000000       ___guard_fids_count        00000000     <absolute>
 0000:00000012       ___safe_se_handler_count   00000012     <absolute>
 0000:00009876       __fltused                  00009876     <absolute>
 0000:00009876       __ldused                   00009876     <absolute>
 0000:00000000       ___ImageBase               10000000     <linker-defined>
 0001:00000510       ??$_Allocate@D@std@@YAPADIPAD@Z 10001510 f i BrowserSupportPlugin.obj
 0001:00000540       ??$addressof@D@std@@YAPADAAD@Z 10001540 f i BrowserSupportPlugin.obj
 0001:00000550       ??$atomic@H@?$QAtomicOpsBySize@$03@@CAPAJPAH@Z 10001550 f i BrowserSupportPlugin.obj
 0001:00000560       ??$construct@PADAAPAD@?$_Wrap_alloc@V?$allocator@D@std@@@std@@QAEXPAPADAAPAD@Z 10001560 f i BrowserSupportPlugin.obj
 0001:00000580       ??$construct@PADAAPAD@?$allocator@D@std@@QAEXPAPADAAPAD@Z 10001580 f i BrowserSupportPlugin.obj
 0001:000005a0       ??$construct@PADAAPAD@?$allocator_traits@V?$allocator@D@std@@@std@@SAXAAV?$allocator@D@1@PAPADAAPAD@Z 100015a0 f i BrowserSupportPlugin.obj
 0001:000005c0       ??$deref@H@?$QAtomicOpsBySize@$03@@SA_NAAH@Z 100015c0 f i BrowserSupportPlugin.obj
 0001:000005e0       ??$destroy@PAD@?$_Wrap_alloc@V?$allocator@D@std@@@std@@QAEXPAPAD@Z 100015e0 f i BrowserSupportPlugin.obj
 0001:000005f0       ??$destroy@PAD@?$allocator@D@std@@QAEXPAPAD@Z 100015f0 f i BrowserSupportPlugin.obj
 0001:00000600       ??$destroy@PAD@?$allocator_traits@V?$allocator@D@std@@@std@@SAXAAV?$allocator@D@1@PAPAD@Z 10001600 f i BrowserSupportPlugin.obj
 0001:00000610       ??$forward@AAPAD@std@@YAAAPADAAPAD@Z 10001610 f i BrowserSupportPlugin.obj
 0001:00000620       ??$load@H@?$QGenericAtomicOps@U?$QAtomicOpsBySize@$03@@@@SAHABH@Z 10001620 f i BrowserSupportPlugin.obj
 0001:00000630       ??0?$QFlags@W4OpenModeFlag@QIODevice@@@@QAE@VQFlag@@@Z 10001630 f i BrowserSupportPlugin.obj
 0001:00000640       ??0?$QFlags@W4OpenModeFlag@QIODevice@@@@QAE@W4OpenModeFlag@QIODevice@@@Z 10001640 f i BrowserSupportPlugin.obj
 0001:00000650       ??0?$QList@VGUrl@U2@@@@QAE@XZ 10001650 f i BrowserSupportPlugin.obj
 0001:00000660       ??0?$QMap@VQString@@VQVariant@@@@QAE@XZ 10001660 f i BrowserSupportPlugin.obj
 0001:00000670       ??0?$_String_alloc@$0A@U?$_String_base_types@DV?$allocator@D@std@@@std@@@std@@QAE@ABV?$allocator@D@1@@Z 10001670 f i BrowserSupportPlugin.obj
 0001:00000690       ??0?$_String_val@U?$_Simple_types@D@std@@@std@@QAE@XZ 10001690 f i BrowserSupportPlugin.obj
 0001:000006b0       ??0?$_Wrap_alloc@V?$allocator@D@std@@@std@@QAE@XZ 100016b0 f i BrowserSupportPlugin.obj
 0001:000006c0       ??0?$allocator@D@std@@QAE@XZ 100016c0 f i BrowserSupportPlugin.obj
 0001:000006d0       ??0?$basic_string@DU?$char_traits@D@std@@V?$allocator@D@2@@std@@QAE@PBD@Z 100016d0 f i BrowserSupportPlugin.obj
 0001:00000730       ??0BrowserSupportPlugin@U2@@QAE@XZ 10001730 f   BrowserSupportPlugin.obj
 0001:00000800       ??0QFlag@@QAE@H@Z          10001800 f i BrowserSupportPlugin.obj
 0001:00000810       ??0_Generic_error_category@std@@QAE@XZ 10001810 f i BrowserSupportPlugin.obj
 0001:00000820       ??0_Ignore@std@@QAE@XZ     10001820 f i BrowserSupportPlugin.obj
 0001:00000830       ??0_Iostream_error_category@std@@QAE@XZ 10001830 f i BrowserSupportPlugin.obj
 0001:00000840       ??0_System_error_category@std@@QAE@XZ 10001840 f i BrowserSupportPlugin.obj
 0001:00000850       ??0error_category@std@@QAE@XZ 10001850 f i BrowserSupportPlugin.obj
 0001:00000860       ??0error_condition@std@@QAE@HABVerror_category@1@@Z 10001860 f i BrowserSupportPlugin.obj
 0001:00000880       ??1?$QList@VGUrl@U2@@@@QAE@XZ 10001880 f i BrowserSupportPlugin.obj
 0001:000008b0       ??1?$QMap@VQString@@VQVariant@@@@QAE@XZ 100018b0 f i BrowserSupportPlugin.obj
 0001:00000900       ??1?$basic_string@DU?$char_traits@D@std@@V?$allocator@D@2@@std@@QAE@XZ 10001900 f i BrowserSupportPlugin.obj
 0001:00000930       ??1BrowserSupportPlugin@U2@@UAE@XZ 10001930 f i BrowserSupportPlugin.obj
 0001:00000940       ??1_Generic_error_category@std@@UAE@XZ 10001940 f i BrowserSupportPlugin.obj
 0001:00000950       ??1_Iostream_error_category@std@@UAE@XZ 10001950 f i BrowserSupportPlugin.obj
 0001:00000960       ??1_System_error_category@std@@UAE@XZ 10001960 f i BrowserSupportPlugin.obj
 0001:00000970       ??1error_category@std@@UAE@XZ 10001970 f i BrowserSupportPlugin.obj
 0001:00000980       ??2@YAPAXIPAX@Z            10001980 f i BrowserSupportPlugin.obj
 0001:00000990       ??3@YAXPAX0@Z              10001990 f i BrowserSupportPlugin.obj
 0001:000009a0       ??6?$QList@VGUrl@U2@@@@QAEAAV0@ABVGUrl@U2@@@Z 100019a0 f i BrowserSupportPlugin.obj
 0001:000009c0       ??8error_category@std@@QBE_NABV01@@Z 100019c0 f i BrowserSupportPlugin.obj
 0001:000009d0       ??8error_condition@std@@QBE_NABV01@@Z 100019d0 f i BrowserSupportPlugin.obj
 0001:000009f0       ??9@YA_NABVQString@@0@Z    100019f0 f i BrowserSupportPlugin.obj
 0001:00000a10       ??BQFlag@@QBEHXZ           10001a10 f i BrowserSupportPlugin.obj
 0001:00000a20       ??U?$QFlags@W4OpenModeFlag@QIODevice@@@@QBE?AV0@W4OpenModeFlag@QIODevice@@@Z 10001a20 f i BrowserSupportPlugin.obj
 0001:00000a40       ??U@YA?AV?$QFlags@W4OpenModeFlag@QIODevice@@@@W4OpenModeFlag@QIODevice@@0@Z 10001a40 f i BrowserSupportPlugin.obj
 0001:00000a50       ??_GBrowserSupportPlugin@U2@@UAEPAXI@Z 10001a50 f i BrowserSupportPlugin.obj
 0001:00000a50       ??_EBrowserSupportPlugin@U2@@UAEPAXI@Z 10001a50 f i BrowserSupportPlugin.obj
 0001:00000a80       ??_GGUrl@U2@@QAEPAXI@Z     10001a80 f i BrowserSupportPlugin.obj
 0001:00000ab0       ??_GLoadRemoteDocumentAndAddToProjectTask@U2@@UAEPAXI@Z 10001ab0 f i BrowserSupportPlugin.obj
 0001:00000ab0       ??_ELoadRemoteDocumentAndAddToProjectTask@U2@@UAEPAXI@Z 10001ab0 f i BrowserSupportPlugin.obj
 0001:00000ae0       ??_GQString@@QAEPAXI@Z     10001ae0 f i BrowserSupportPlugin.obj
 0001:00000b10       ??_GQVariant@@QAEPAXI@Z    10001b10 f i BrowserSupportPlugin.obj
 0001:00000b40       ??_G_Generic_error_category@std@@UAEPAXI@Z 10001b40 f i BrowserSupportPlugin.obj
 0001:00000b40       ??_E_Generic_error_category@std@@UAEPAXI@Z 10001b40 f i BrowserSupportPlugin.obj
 0001:00000b70       ??_G_Iostream_error_category@std@@UAEPAXI@Z 10001b70 f i BrowserSupportPlugin.obj
 0001:00000b70       ??_E_Iostream_error_category@std@@UAEPAXI@Z 10001b70 f i BrowserSupportPlugin.obj
 0001:00000ba0       ??_G_System_error_category@std@@UAEPAXI@Z 10001ba0 f i BrowserSupportPlugin.obj
 0001:00000ba0       ??_E_System_error_category@std@@UAEPAXI@Z 10001ba0 f i BrowserSupportPlugin.obj
 0001:00000bd0       ??_Gerror_category@std@@UAEPAXI@Z 10001bd0 f i BrowserSupportPlugin.obj
 0001:00000bd0       ??_Eerror_category@std@@UAEPAXI@Z 10001bd0 f i BrowserSupportPlugin.obj
 0001:00000c00       ?_Copy@?$basic_string@DU?$char_traits@D@std@@V?$allocator@D@2@@std@@QAEXII@Z 10001c00 f i BrowserSupportPlugin.obj
 0001:00000d50       ?_Eos@?$basic_string@DU?$char_traits@D@std@@V?$allocator@D@2@@std@@QAEXI@Z 10001d50 f i BrowserSupportPlugin.obj
 0001:00000d80       ?_Getal@?$_String_alloc@$0A@U?$_String_base_types@DV?$allocator@D@std@@@std@@@std@@QBE?AU?$_Wrap_alloc@V?$allocator@D@std@@@2@XZ 10001d80 f i BrowserSupportPlugin.obj
 0001:00000d90       ?_Grow@?$basic_string@DU?$char_traits@D@std@@V?$allocator@D@2@@std@@QAE_NI_N@Z 10001d90 f i BrowserSupportPlugin.obj
 0001:00000e40       ?_Inside@?$basic_string@DU?$char_traits@D@std@@V?$allocator@D@2@@std@@QAE_NPBD@Z 10001e40 f i BrowserSupportPlugin.obj
 0001:00000e80       ?_Myptr@?$_String_val@U?$_Simple_types@D@std@@@std@@QAEPADXZ 10001e80 f i BrowserSupportPlugin.obj
 0001:00000e90       ?_Myptr@?$_String_val@U?$_Simple_types@D@std@@@std@@QBEPBDXZ 10001e90 f i BrowserSupportPlugin.obj
 0001:00000ea0       ?_Tidy@?$basic_string@DU?$char_traits@D@std@@V?$allocator@D@2@@std@@QAEX_NI@Z 10001ea0 f i BrowserSupportPlugin.obj
 0001:00000ef0       ?_Xlen@?$basic_string@DU?$char_traits@D@std@@V?$allocator@D@2@@std@@QBEXXZ 10001ef0 f i BrowserSupportPlugin.obj
 0001:00000f00       ?_Xran@?$basic_string@DU?$char_traits@D@std@@V?$allocator@D@2@@std@@QBEXXZ 10001f00 f i BrowserSupportPlugin.obj
 0001:00000f10       ?allocate@?$_Wrap_alloc@V?$allocator@D@std@@@std@@QAEPADI@Z 10001f10 f i BrowserSupportPlugin.obj
 0001:00000f40       ?allocate@?$allocator@D@std@@QAEPADI@Z 10001f40 f i BrowserSupportPlugin.obj
 0001:00000f70       ?append@?$QList@VGUrl@U2@@@@QAEXABVGUrl@U2@@@Z 10001f70 f i BrowserSupportPlugin.obj
 0001:00001050       ?assign@?$basic_string@DU?$char_traits@D@std@@V?$allocator@D@2@@std@@QAEAAV12@ABV12@II@Z 10002050 f i BrowserSupportPlugin.obj
 0001:00001170       ?assign@?$basic_string@DU?$char_traits@D@std@@V?$allocator@D@2@@std@@QAEAAV12@PBD@Z 10002170 f i BrowserSupportPlugin.obj
 0001:000011b0       ?assign@?$basic_string@DU?$char_traits@D@std@@V?$allocator@D@2@@std@@QAEAAV12@PBDI@Z 100021b0 f i BrowserSupportPlugin.obj
 0001:000012b0       ?assign@?$char_traits@D@std@@SAXAADABD@Z 100022b0 f i BrowserSupportPlugin.obj
 0001:000012c0       ?category@error_code@std@@QBEABVerror_category@2@XZ 100022c0 f i BrowserSupportPlugin.obj
 0001:000012d0       ?category@error_condition@std@@QBEABVerror_category@2@XZ 100022d0 f i BrowserSupportPlugin.obj
 0001:000012e0       ?copy@?$char_traits@D@std@@SAPADPADPBDI@Z 100022e0 f i BrowserSupportPlugin.obj
 0001:00001300       ?dealloc@?$QList@VGUrl@U2@@@@AAEXPAUData@QListData@@@Z 10002300 f i BrowserSupportPlugin.obj
 0001:00001360       ?deallocate@?$_Wrap_alloc@V?$allocator@D@std@@@std@@QAEXPADI@Z 10002360 f i BrowserSupportPlugin.obj
 0001:00001380       ?deallocate@?$allocator@D@std@@QAEXPADI@Z 10002380 f i BrowserSupportPlugin.obj
 0001:000013a0       ?default_error_condition@_System_error_category@std@@UBE?AVerror_condition@2@H@Z 100023a0 f i BrowserSupportPlugin.obj
 0001:000013e0       ?default_error_condition@error_category@std@@UBE?AVerror_condition@2@H@Z 100023e0 f i BrowserSupportPlugin.obj
 0001:00001400       ?deref@?$QBasicAtomicInteger@H@@QAE_NXZ 10002400 f i BrowserSupportPlugin.obj
 0001:00001410       ?deref@RefCount@QtPrivate@@QAE_NXZ 10002410 f i BrowserSupportPlugin.obj
 0001:00001430       ?destroy@?$QMapData@VQString@@VQVariant@@@@QAEXXZ 10002430 f i BrowserSupportPlugin.obj
 0001:00001460       ?destroySubTree@?$QMapNode@VQString@@VQVariant@@@@QAEXXZ 10002460 f i BrowserSupportPlugin.obj
 0001:000014a0       ?detach_helper_grow@?$QList@VGUrl@U2@@@@AAEPAUNode@1@HH@Z 100024a0 f i BrowserSupportPlugin.obj
 0001:000015f0       ?equivalent@error_category@std@@UBE_NABVerror_code@2@H@Z 100025f0 f i BrowserSupportPlugin.obj
 0001:00001610       ?equivalent@error_category@std@@UBE_NHABVerror_condition@2@@Z 10002610 f i BrowserSupportPlugin.obj
 0001:00001650       ?erase@?$basic_string@DU?$char_traits@D@std@@V?$allocator@D@2@@std@@QAEAAV12@I@Z 10002650 f i BrowserSupportPlugin.obj
 0001:00001690       ?erase@?$basic_string@DU?$char_traits@D@std@@V?$allocator@D@2@@std@@QAEAAV12@II@Z 10002690 f i BrowserSupportPlugin.obj
 0001:00001730       ?generic_category@std@@YAABVerror_category@1@XZ 10002730 f i BrowserSupportPlugin.obj
 0001:00001740       ?isShared@RefCount@QtPrivate@@QBE_NXZ 10002740 f i BrowserSupportPlugin.obj
 0001:00001760       ?leftNode@?$QMapNode@VQString@@VQVariant@@@@QBEPAU1@XZ 10002760 f i BrowserSupportPlugin.obj
 0001:00001770       ?length@?$char_traits@D@std@@SAIPBD@Z 10002770 f i BrowserSupportPlugin.obj
 0001:00001790       ?load@?$QBasicAtomicInteger@H@@QBEHXZ 10002790 f i BrowserSupportPlugin.obj
 0001:000017a0       ?max_size@?$_Wrap_alloc@V?$allocator@D@std@@@std@@QBEIXZ 100027a0 f i BrowserSupportPlugin.obj
 0001:000017b0       ?max_size@?$allocator@D@std@@QBEIXZ 100027b0 f i BrowserSupportPlugin.obj
 0001:000017c0       ?max_size@?$allocator_traits@V?$allocator@D@std@@@std@@SAIABV?$allocator@D@2@@Z 100027c0 f i BrowserSupportPlugin.obj
 0001:000017d0       ?max_size@?$basic_string@DU?$char_traits@D@std@@V?$allocator@D@2@@std@@QBEIXZ 100027d0 f i BrowserSupportPlugin.obj
 0001:000017e0       ?message@_Generic_error_category@std@@UBE?AV?$basic_string@DU?$char_traits@D@std@@V?$allocator@D@2@@2@H@Z 100027e0 f i BrowserSupportPlugin.obj
 0001:00001860       ?message@_Iostream_error_category@std@@UBE?AV?$basic_string@DU?$char_traits@D@std@@V?$allocator@D@2@@2@H@Z 10002860 f i BrowserSupportPlugin.obj
 0001:000018b0       ?message@_System_error_category@std@@UBE?AV?$basic_string@DU?$char_traits@D@std@@V?$allocator@D@2@@2@H@Z 100028b0 f i BrowserSupportPlugin.obj
 0001:00001930       ?move@?$char_traits@D@std@@SAPADPADPBDI@Z 10002930 f i BrowserSupportPlugin.obj
 0001:00001950       ?name@_Generic_error_category@std@@UBEPBDXZ 10002950 f i BrowserSupportPlugin.obj
 0001:00001960       ?name@_Iostream_error_category@std@@UBEPBDXZ 10002960 f i BrowserSupportPlugin.obj
 0001:00001970       ?name@_System_error_category@std@@UBEPBDXZ 10002970 f i BrowserSupportPlugin.obj
 0001:00001980       ?node_construct@?$QList@VGUrl@U2@@@@AAEXPAUNode@1@ABVGUrl@U2@@@Z 10002980 f i BrowserSupportPlugin.obj
 0001:00001a00       ?node_copy@?$QList@VGUrl@U2@@@@AAEXPAUNode@1@00@Z 10002a00 f i BrowserSupportPlugin.obj
 0001:00001ad0       ?node_destruct@?$QList@VGUrl@U2@@@@AAEXPAUNode@1@0@Z 10002ad0 f i BrowserSupportPlugin.obj
 0001:00001b10       ?node_destruct@?$QList@VGUrl@U2@@@@AAEXPAUNode@1@@Z 10002b10 f i BrowserSupportPlugin.obj
 0001:00001b40       ?rightNode@?$QMapNode@VQString@@VQVariant@@@@QBEPAU1@XZ 10002b40 f i BrowserSupportPlugin.obj
 0001:00001b50       ?root@?$QMapData@VQString@@VQVariant@@@@QBEPAU?$QMapNode@VQString@@VQVariant@@@@XZ 10002b50 f i BrowserSupportPlugin.obj
 0001:00001b60       ?saveToTmp@BrowserSupportPlugin@U2@@IAE?AVQString@@AAV3@@Z 10002b60 f   BrowserSupportPlugin.obj
 0001:00001cc0       ?size@?$basic_string@DU?$char_traits@D@std@@V?$allocator@D@2@@std@@QBEIXZ 10002cc0 f i BrowserSupportPlugin.obj
 0001:00001cd0       ?sl_clipboardCheck@BrowserSupportPlugin@U2@@IAEXXZ 10002cd0 f   BrowserSupportPlugin.obj
 0001:00002530       ?system_category@std@@YAABVerror_category@1@XZ 10003530 f i BrowserSupportPlugin.obj
 0001:00002540       ?tr@BrowserSupportPlugin@U2@@SA?AVQString@@PBD0H@Z 10003540 f i BrowserSupportPlugin.obj
 0001:00002570       ?value@error_code@std@@QBEHXZ 10003570 f i BrowserSupportPlugin.obj
 0001:00002580       ?value@error_condition@std@@QBEHXZ 10003580 f i BrowserSupportPlugin.obj
 0001:00002590       _hypot                     10003590 f i BrowserSupportPlugin.obj
 0001:000025c0       _ugene_plugin_init         100035c0 f   BrowserSupportPlugin.obj
 0001:000025f0       ??C?$QScopedPointer@VQObjectData@@U?$QScopedPointerDeleter@VQObjectData@@@@@@QBEPAVQObjectData@@XZ 100035f0 f i moc_BrowserSupportPlugin.obj
 0001:00002600       ?metaObject@BrowserSupportPlugin@U2@@UBEPBUQMetaObject@@XZ 10003600 f   moc_BrowserSupportPlugin.obj
 0001:00002620       ?qt_metacall@BrowserSupportPlugin@U2@@UAEHW4Call@QMetaObject@@HPAPAX@Z 10003620 f   moc_BrowserSupportPlugin.obj
 0001:00002680       ?qt_metacast@BrowserSupportPlugin@U2@@UAEPAXPBD@Z 10003680 f   moc_BrowserSupportPlugin.obj
 0001:000026e0       ?qt_noop@@YAXXZ            100036e0 f i moc_BrowserSupportPlugin.obj
 0001:000026f0       ?qt_static_metacall@BrowserSupportPlugin@U2@@CAXPAVQObject@@W4Call@QMetaObject@@HPAPAX@Z 100036f0 f   moc_BrowserSupportPlugin.obj
 0001:0000270a       ?getProjectLoader@AppContext@U2@@SAPAVProjectLoader@2@XZ 1000370a f   U2Core:U2Core.dll
 0001:00002710       ?getAppSettings@AppContext@U2@@SAPAVAppSettings@2@XZ 10003710 f   U2Core:U2Core.dll
 0001:00002716       ?getMainWindow@AppContext@U2@@SAPAVMainWindow@2@XZ 10003716 f   U2Core:U2Core.dll
 0001:0000271c       ?getTaskScheduler@AppContext@U2@@SAPAVTaskScheduler@2@XZ 1000371c f   U2Core:U2Core.dll
 0001:00002722       ??0Logger@U2@@QAE@ABVQString@@@Z 10003722 f   U2Core:U2Core.dll
 0001:00002728       ??1Logger@U2@@UAE@XZ       10003728 f   U2Core:U2Core.dll
 0001:0000272e       ??0GUrl@U2@@QAE@ABVQString@@W4GUrlType@1@@Z 1000372e f   U2Core:U2Core.dll
 0001:00002734       ??0GUrl@U2@@QAE@ABV01@@Z   10003734 f   U2Core:U2Core.dll
 0001:0000273a       ??1GUrl@U2@@QAE@XZ         1000373a f   U2Core:U2Core.dll
 0001:00002740       ??1GCounter@U2@@UAE@XZ     10003740 f   U2Core:U2Core.dll
 0001:00002746       ??0GReportableCounter@U2@@QAE@ABVQString@@0N@Z 10003746 f   U2Core:U2Core.dll
 0001:0000274c       ??1SimpleEventCounter@U2@@UAE@XZ 1000374c f   U2Core:U2Core.dll
 0001:00002752       ?getCurrentProcessTemporaryDirPath@UserAppsSettings@U2@@QBE?AVQString@@ABV3@@Z 10003752 f   U2Core:U2Core.dll
 0001:00002758       ?prepareDownloadDirectory@BaseLoadRemoteDocumentTask@U2@@SA_NAAVQString@@@Z 10003758 f   U2Core:U2Core.dll
 0001:0000275e       ?getDefaultDownloadDirectory@BaseLoadRemoteDocumentTask@U2@@SA?AVQString@@XZ 1000375e f   U2Core:U2Core.dll
 0001:00002764       ??0U2OpStatus2Log@U2@@QAE@W4LogLevel@1@@Z 10003764 f   U2Core:U2Core.dll
 0001:0000276a       ??1U2OpStatus2Log@U2@@UAE@XZ 1000376a f   U2Core:U2Core.dll
 0001:00002770       ?prepareTmpFileLocation@GUrlUtils@U2@@SA?AVQString@@ABV3@00AAVU2OpStatus@2@@Z 10003770 f   U2Core:U2Core.dll
 0001:00002776       ??0Plugin@U2@@QAE@ABVQString@@0_NW4PluginState@1@@Z 10003776 f   U2Core:U2Core.dll
 0001:0000277c       ??1Plugin@U2@@UAE@XZ       1000377c f   U2Core:U2Core.dll
 0001:00002782       ?cleanup@Task@U2@@UAEXXZ   10003782 f   U2Core:U2Core.dll
 0001:00002788       ?getNumParallelSubtasks@Task@U2@@UBEHXZ 10003788 f   U2Core:U2Core.dll
 0001:0000278e       ?getParentTask@Task@U2@@UBEPAV12@XZ 1000378e f   U2Core:U2Core.dll
 0001:00002794       ?getSubtaskWithErrors@Task@U2@@UBEPAV12@XZ 10003794 f   U2Core:U2Core.dll
 0001:0000279a       ?getTaskId@Task@U2@@UBE_JXZ 1000379a f   U2Core:U2Core.dll
 0001:000027a0       ?getTopLevelParentTask@Task@U2@@UAEPAV12@XZ 100037a0 f   U2Core:U2Core.dll
 0001:000027a6       ?getWarnings@Task@U2@@UBE?AVQStringList@@XZ 100037a6 f   U2Core:U2Core.dll
 0001:000027ac       ?hasSubtasksWithErrors@Task@U2@@UBE_NXZ 100037ac f   U2Core:U2Core.dll
 0001:000027b2       ?hasWarning@Task@U2@@UBE_NXZ 100037b2 f   U2Core:U2Core.dll
 0001:000027b8       ?isNotificationReport@Task@U2@@UBE_NXZ 100037b8 f   U2Core:U2Core.dll
 0001:000027be       ?isReportingEnabled@Task@U2@@UBE_NXZ 100037be f   U2Core:U2Core.dll
 0001:000027c4       ?isReportingSupported@Task@U2@@UBE_NXZ 100037c4 f   U2Core:U2Core.dll
 0001:000027ca       ?isTopLevelTask@Task@U2@@UBE_NXZ 100037ca f   U2Core:U2Core.dll
 0001:000027d0       ?propagateSubtaskError@Task@U2@@UAE_NXZ 100037d0 f   U2Core:U2Core.dll
 0001:000027d6       ?report@Task@U2@@UAE?AW4ReportResult@12@XZ 100037d6 f   U2Core:U2Core.dll
 0001:000027dc       ?run@Task@U2@@UAEXXZ       100037dc f   U2Core:U2Core.dll
 0001:000027e2       ?setCollectChildrensWarningsFlag@Task@U2@@UAEX_N@Z 100037e2 f   U2Core:U2Core.dll
 0001:000027e8       ?setNoAutoDelete@Task@U2@@UAEX_N@Z 100037e8 f   U2Core:U2Core.dll
 0001:000027ee       ?setNotificationReport@Task@U2@@UAEX_N@Z 100037ee f   U2Core:U2Core.dll
 0001:000027f4       ?setReportingEnabled@Task@U2@@UAEX_N@Z 100037f4 f   U2Core:U2Core.dll
 0001:000027fa       ?setReportingSupported@Task@U2@@UAEX_N@Z 100037fa f   U2Core:U2Core.dll
 0001:00002800       ?qt_metacast@Plugin@U2@@UAEPAXPBD@Z 10003800 f   U2Core:U2Core.dll
 0001:00002806       ?qt_metacall@Plugin@U2@@UAEHW4Call@QMetaObject@@HPAPAX@Z 10003806 f   U2Core:U2Core.dll
 0001:0000280c       ??0LoadRemoteDocumentAndAddToProjectTask@U2@@QAE@ABVQString@@000ABV?$QMap@VQString@@VQVariant@@@@W4LoadRemoteDocumentMode@1@@Z 1000380c f   U2Gui:U2Gui.dll
 0001:00002812       ??1LoadRemoteDocumentAndAddToProjectTask@U2@@UAE@XZ 10003812 f   U2Gui:U2Gui.dll
 0001:00002818       ?generateReport@LoadRemoteDocumentAndAddToProjectTask@U2@@UBE?AVQString@@XZ 10003818 f   U2Gui:U2Gui.dll
 0001:0000281e       ?metaObject@LoadRemoteDocumentAndAddToProjectTask@U2@@UBEPBUQMetaObject@@XZ 1000381e f   U2Gui:U2Gui.dll
 0001:00002824       ?onSubTaskFinished@LoadRemoteDocumentAndAddToProjectTask@U2@@MAE?AV?$QList@PAVTask@U2@@@@PAVTask@2@@Z 10003824 f   U2Gui:U2Gui.dll
 0001:0000282a       ?prepare@LoadRemoteDocumentAndAddToProjectTask@U2@@UAEXXZ 1000382a f   U2Gui:U2Gui.dll
 0001:00002830       ?qt_metacall@LoadRemoteDocumentAndAddToProjectTask@U2@@UAEHW4Call@QMetaObject@@HPAPAX@Z 10003830 f   U2Gui:U2Gui.dll
 0001:00002836       ?qt_metacast@LoadRemoteDocumentAndAddToProjectTask@U2@@UAEPAXPBD@Z 10003836 f   U2Gui:U2Gui.dll
 0001:0000283c       ?text@QClipboard@@QBE?AVQString@@W4Mode@1@@Z 1000383c f   Qt5Gui:Qt5Gui.dll
 0001:00002842       ?setText@QClipboard@@QAEXABVQString@@W4Mode@1@@Z 10003842 f   Qt5Gui:Qt5Gui.dll
 0001:00002848       ?clipboard@QGuiApplication@@SAPAVQClipboard@@XZ 10003848 f   Qt5Gui:Qt5Gui.dll
 0001:0000284e       ??0QString@@QAE@XZ         1000384e f   Qt5Core:Qt5Core.dll
 0001:00002854       ??0QString@@QAE@PBVQChar@@H@Z 10003854 f   Qt5Core:Qt5Core.dll
 0001:0000285a       ??1QString@@QAE@XZ         1000385a f   Qt5Core:Qt5Core.dll
 0001:00002860       ??4QString@@QAEAAV0@ABV0@@Z 10003860 f   Qt5Core:Qt5Core.dll
 0001:00002866       ??4QString@@QAEAAV0@$$QAV0@@Z 10003866 f   Qt5Core:Qt5Core.dll
 0001:0000286c       ?data@QString@@QAEPAVQChar@@XZ 1000386c f   Qt5Core:Qt5Core.dll
 0001:00002872       ?indexOf@QString@@QBEHABV1@HW4CaseSensitivity@Qt@@@Z 10003872 f   Qt5Core:Qt5Core.dll
 0001:00002878       ?left@QString@@QBE?AV1@H@Z 10003878 f   Qt5Core:Qt5Core.dll
 0001:0000287e       ?startsWith@QString@@QBE_NABV1@W4CaseSensitivity@Qt@@@Z 1000387e f   Qt5Core:Qt5Core.dll
 0001:00002884       ?trimmed@QString@@QBE?AV1@XZ 10003884 f   Qt5Core:Qt5Core.dll
 0001:0000288a       ?simplified@QString@@QBE?AV1@XZ 1000388a f   Qt5Core:Qt5Core.dll
 0001:00002890       ??8@YA_NABVQString@@0@Z    10003890 f   Qt5Core:Qt5Core.dll
 0001:00002896       ?fromAscii_helper@QString@@CAPAU?$QTypedArrayData@G@@PBDH@Z 10003896 f   Qt5Core:Qt5Core.dll
 0001:0000289c       ?tr@QMetaObject@@QBE?AVQString@@PBD0H@Z 1000389c f   Qt5Core:Qt5Core.dll
 0001:000028a2       ??1Connection@QMetaObject@@QAE@XZ 100038a2 f   Qt5Core:Qt5Core.dll
 0001:000028a8       ?detach_grow@QListData@@QAEPAUData@1@PAHH@Z 100038a8 f   Qt5Core:Qt5Core.dll
 0001:000028ae       ?dispose@QListData@@SAXPAUData@1@@Z 100038ae f   Qt5Core:Qt5Core.dll
 0001:000028b4       ?append@QListData@@QAEPAPAXXZ 100038b4 f   Qt5Core:Qt5Core.dll
 0001:000028ba       ?connect@QObject@@QBE?AVConnection@QMetaObject@@PBV1@PBD1W4ConnectionType@Qt@@@Z 100038ba f   Qt5Core:Qt5Core.dll
 0001:000028c0       ??0QFile@@QAE@ABVQString@@@Z 100038c0 f   Qt5Core:Qt5Core.dll
 0001:000028c6       ??1QFile@@UAE@XZ           100038c6 f   Qt5Core:Qt5Core.dll
 0001:000028cc       ?open@QFile@@UAE_NV?$QFlags@W4OpenModeFlag@QIODevice@@@@@Z 100038cc f   Qt5Core:Qt5Core.dll
 0001:000028d2       ?toNativeSeparators@QDir@@SA?AVQString@@ABV2@@Z 100038d2 f   Qt5Core:Qt5Core.dll
 0001:000028d8       ?freeTree@QMapDataBase@@QAEXPAUQMapNodeBase@@H@Z 100038d8 f   Qt5Core:Qt5Core.dll
 0001:000028de       ?freeData@QMapDataBase@@SAXPAU1@@Z 100038de f   Qt5Core:Qt5Core.dll
 0001:000028e4       ??1QVariant@@QAE@XZ        100038e4 f   Qt5Core:Qt5Core.dll
 0001:000028ea       ??0QTextStream@@QAE@PAVQIODevice@@@Z 100038ea f   Qt5Core:Qt5Core.dll
 0001:000028f0       ??1QTextStream@@UAE@XZ     100038f0 f   Qt5Core:Qt5Core.dll
 0001:000028f6       ??6QTextStream@@QAEAAV0@ABVQString@@@Z 100038f6 f   Qt5Core:Qt5Core.dll
 0001:000028fc       ?childEvent@QObject@@MAEXPAVQChildEvent@@@Z 100038fc f   Qt5Core:Qt5Core.dll
 0001:00002902       ?connectNotify@QObject@@MAEXABVQMetaMethod@@@Z 10003902 f   Qt5Core:Qt5Core.dll
 0001:00002908       ?customEvent@QObject@@MAEXPAVQEvent@@@Z 10003908 f   Qt5Core:Qt5Core.dll
 0001:0000290e       ?disconnectNotify@QObject@@MAEXABVQMetaMethod@@@Z 1000390e f   Qt5Core:Qt5Core.dll
 0001:00002914       ?event@QObject@@UAE_NPAVQEvent@@@Z 10003914 f   Qt5Core:Qt5Core.dll
 0001:0000291a       ?eventFilter@QObject@@UAE_NPAV1@PAVQEvent@@@Z 1000391a f   Qt5Core:Qt5Core.dll
 0001:00002920       ?timerEvent@QObject@@MAEXPAVQTimerEvent@@@Z 10003920 f   Qt5Core:Qt5Core.dll
 0001:00002926       ?dynamicMetaObject@QObjectData@@QBEPAUQMetaObject@@XZ 10003926 f   Qt5Core:Qt5Core.dll
 0001:0000292c       ?_Xbad_alloc@std@@YAXXZ    1000392c f   msvcprt:MSVCP120.dll
 0001:00002932       ?_Xlength_error@std@@YAXPBD@Z 10003932 f   msvcprt:MSVCP120.dll
 0001:00002938       ?_Xout_of_range@std@@YAXPBD@Z 10003938 f   msvcprt:MSVCP120.dll
 0001:0000293e       ?_Syserror_map@std@@YAPBDH@Z 1000393e f   msvcprt:MSVCP120.dll
 0001:00002944       ?_Winerror_map@std@@YAPBDH@Z 10003944 f   msvcprt:MSVCP120.dll
 0001:0000294a       __purecall                 1000394a f   MSVCRT:MSVCR120.dll
 0001:00002950       ??2@YAPAXI@Z               10003950 f   MSVCRT:MSVCR120.dll
 0001:00002956       ??3@YAXPAX@Z               10003956 f   MSVCRT:MSVCR120.dll
 0001:0000295c       ___atonexitinit            1000395c f   MSVCRT:atonexit.obj
 0001:00002998       __onexit                   10003998 f   MSVCRT:atonexit.obj
 0001:00002a41       _atexit                    10003a41 f   MSVCRT:atonexit.obj
 0001:00002a56       _memmove                   10003a56 f   MSVCRT:MSVCR120.dll
 0001:00002a5c       __hypot                    10003a5c f   MSVCRT:MSVCR120.dll
 0001:00002a62       @__security_check_cookie@4 10003a62 f   MSVCRT:secchk.obj
 0001:00002a72       __CxxThrowException@8      10003a72 f   MSVCRT:MSVCR120.dll
 0001:00002a78       ___CxxFrameHandler3        10003a78 f   MSVCRT:MSVCR120.dll
 0001:00002a7e       _memcpy                    10003a7e f   MSVCRT:MSVCR120.dll
 0001:00002a84       ??0type_info@@AAE@ABV0@@Z  10003a84 f   MSVCRT:ti_inst.obj
 0001:00002a8f       ??4type_info@@AAEAAV0@ABV0@@Z 10003a8f f   MSVCRT:ti_inst.obj
 0001:00002a94       ??_Etype_info@@UAEPAXI@Z   10003a94 f i MSVCRT:ti_inst.obj
 0001:00002b2c       _NtCurrentTeb              10003b2c f i MSVCRT:crtdll.obj
 0001:00002b33       __CRT_INIT@12              10003b33 f   MSVCRT:crtdll.obj
 0001:00002d2a       __DllMainCRTStartup@12     10003d2a f   MSVCRT:crtdll.obj
 0001:00002e80       __lock                     10003e80 f   MSVCRT:MSVCR120.dll
 0001:00002e86       __unlock                   10003e86 f   MSVCRT:MSVCR120.dll
 0001:00002e8c       __calloc_crt               10003e8c f   MSVCRT:MSVCR120.dll
 0001:00002e92       ___dllonexit               10003e92 f   MSVCRT:MSVCR120.dll
 0001:00002ea0       __SEH_prolog4              10003ea0 f   MSVCRT:sehprolg4.obj
 0001:00002ee5       __SEH_epilog4              10003ee5 f   MSVCRT:sehprolg4.obj
 0001:00002ef9       __except_handler4          10003ef9 f   MSVCRT:chandler4gs.obj
 0001:00002f1c       ___raise_securityfailure   10003f1c f   MSVCRT:gs_report.obj
 0001:00002f59       ___report_gsfailure        10003f59 f   MSVCRT:gs_report.obj
 0001:00003054       ___report_rangecheckfailure 10004054 f   MSVCRT:gs_report.obj
 0001:00003060       ___report_securityfailure  10004060 f   MSVCRT:gs_report.obj
 0001:00003130       ___report_securityfailureEx 10004130 f   MSVCRT:gs_report.obj
 0001:00003246       ??_M@YGXPAXIHP6EX0@Z@Z     10004246 f   MSVCRT:ehvecdtr.obj
 0001:000032ce       ?__ArrayUnwind@@YGXPAXIHP6EX0@Z@Z 100042ce f   MSVCRT:ehvecdtr.obj
 0001:0000332c       ??1type_info@@UAE@XZ       1000432c f   MSVCRT:MSVCR120.dll
 0001:00003332       ___CppXcptFilter           10004332 f   MSVCRT:MSVCR120.dll
 0001:00003338       __amsg_exit                10004338 f   MSVCRT:MSVCR120.dll
 0001:00003340       __FindPESection            10004340 f   MSVCRT:pesect.obj
 0001:00003390       __IsNonwritableInCurrentImage 10004390 f   MSVCRT:pesect.obj
 0001:00003450       __ValidateImageBase        10004450 f   MSVCRT:pesect.obj
 0001:00003482       _free                      10004482 f   MSVCRT:MSVCR120.dll
 0001:00003488       ___security_init_cookie    10004488 f   MSVCRT:gs_support.obj
 0001:00003524       _DllMain@12                10004524 f   MSVCRT:dllmain.obj
 0001:00003546       __malloc_crt               10004546 f   MSVCRT:MSVCR120.dll
 0001:0000354c       __RTC_Initialize           1000454c f   MSVCRT:initsect.obj
 0001:0000356c       __RTC_Terminate            1000456c f   MSVCRT:initsect.obj
 0001:0000358c       __initterm                 1000458c f   MSVCRT:MSVCR120.dll
 0001:00003592       __initterm_e               10004592 f   MSVCRT:MSVCR120.dll
 0001:00003598       ___clean_type_info_names   10004598 f   MSVCRT:tncleanup.obj
 0001:000035a4       __except_handler4_common   100045a4 f   MSVCRT:MSVCR120.dll
 0001:000035aa       __crt_debugger_hook        100045aa f   MSVCRT:MSVCR120.dll
 0001:000035b0       ___crtUnhandledException   100045b0 f   MSVCRT:MSVCR120.dll
 0001:000035b6       ___crtTerminateProcess     100045b6 f   MSVCRT:MSVCR120.dll
 0001:000035bc       ?terminate@@YAXXZ          100045bc f   MSVCRT:MSVCR120.dll
 0001:000035c2       ___clean_type_info_names_internal 100045c2 f   MSVCRT:MSVCR120.dll
 0001:000035c8       _EncodePointer@4           100045c8 f   kernel32:KERNEL32.dll
 0001:000035ce       _DecodePointer@4           100045ce f   kernel32:KERNEL32.dll
 0001:000035d4       _IsDebuggerPresent@0       100045d4 f   kernel32:KERNEL32.dll
 0001:000035da       _IsProcessorFeaturePresent@4 100045da f   kernel32:KERNEL32.dll
 0001:000035e0       _QueryPerformanceCounter@4 100045e0 f   kernel32:KERNEL32.dll
 0001:000035e6       _GetCurrentProcessId@0     100045e6 f   kernel32:KERNEL32.dll
 0001:000035ec       _GetCurrentThreadId@0      100045ec f   kernel32:KERNEL32.dll
 0001:000035f2       _GetSystemTimeAsFileTime@4 100045f2 f   kernel32:KERNEL32.dll
 0001:000035f8       _DisableThreadLibraryCalls@4 100045f8 f   kernel32:KERNEL32.dll
 0002:00000000       __imp__DisableThreadLibraryCalls@4 10005000     kernel32:KERNEL32.dll
 0002:00000004       __imp__GetSystemTimeAsFileTime@4 10005004     kernel32:KERNEL32.dll
 0002:00000008       __imp__GetCurrentThreadId@0 10005008     kernel32:KERNEL32.dll
 0002:0000000c       __imp__GetCurrentProcessId@0 1000500c     kernel32:KERNEL32.dll
 0002:00000010       __imp__QueryPerformanceCounter@4 10005010     kernel32:KERNEL32.dll
 0002:00000014       __imp__IsProcessorFeaturePresent@4 10005014     kernel32:KERNEL32.dll
 0002:00000018       __imp__IsDebuggerPresent@0 10005018     kernel32:KERNEL32.dll
 0002:0000001c       __imp__DecodePointer@4     1000501c     kernel32:KERNEL32.dll
 0002:00000020       __imp__EncodePointer@4     10005020     kernel32:KERNEL32.dll
 0002:00000024       \177KERNEL32_NULL_THUNK_DATA 10005024     kernel32:KERNEL32.dll
 0002:00000028       __imp_?_Xlength_error@std@@YAXPBD@Z 10005028     msvcprt:MSVCP120.dll
 0002:0000002c       __imp_?_Xout_of_range@std@@YAXPBD@Z 1000502c     msvcprt:MSVCP120.dll
 0002:00000030       __imp_?_Syserror_map@std@@YAPBDH@Z 10005030     msvcprt:MSVCP120.dll
 0002:00000034       __imp_?_Winerror_map@std@@YAPBDH@Z 10005034     msvcprt:MSVCP120.dll
 0002:00000038       __imp_?_Xbad_alloc@std@@YAXXZ 10005038     msvcprt:MSVCP120.dll
 0002:0000003c       \177MSVCP120_NULL_THUNK_DATA 1000503c     msvcprt:MSVCP120.dll
 0002:00000040       __imp___initterm_e         10005040     MSVCRT:MSVCR120.dll
 0002:00000044       __imp___initterm           10005044     MSVCRT:MSVCR120.dll
 0002:00000048       __imp___malloc_crt         10005048     MSVCRT:MSVCR120.dll
 0002:0000004c       __imp__free                1000504c     MSVCRT:MSVCR120.dll
 0002:00000050       __imp___except_handler4_common 10005050     MSVCRT:MSVCR120.dll
 0002:00000054       __imp____CppXcptFilter     10005054     MSVCRT:MSVCR120.dll
 0002:00000058       __imp_??1type_info@@UAE@XZ 10005058     MSVCRT:MSVCR120.dll
 0002:0000005c       __imp___onexit             1000505c     MSVCRT:MSVCR120.dll
 0002:00000060       __imp____dllonexit         10005060     MSVCRT:MSVCR120.dll
 0002:00000064       __imp___calloc_crt         10005064     MSVCRT:MSVCR120.dll
 0002:00000068       __imp___unlock             10005068     MSVCRT:MSVCR120.dll
 0002:0000006c       __imp___lock               1000506c     MSVCRT:MSVCR120.dll
 0002:00000070       __imp__memcpy              10005070     MSVCRT:MSVCR120.dll
 0002:00000074       __imp____CxxFrameHandler3  10005074     MSVCRT:MSVCR120.dll
 0002:00000078       __imp___CxxThrowException@8 10005078     MSVCRT:MSVCR120.dll
 0002:0000007c       __imp___hypot              1000507c     MSVCRT:MSVCR120.dll
 0002:00000080       __imp__memmove             10005080     MSVCRT:MSVCR120.dll
 0002:00000084       __imp_??3@YAXPAX@Z         10005084     MSVCRT:MSVCR120.dll
 0002:00000088       __imp_??2@YAPAXI@Z         10005088     MSVCRT:MSVCR120.dll
 0002:0000008c       __imp___purecall           1000508c     MSVCRT:MSVCR120.dll
 0002:00000090       __imp___crt_debugger_hook  10005090     MSVCRT:MSVCR120.dll
 0002:00000094       __imp____crtUnhandledException 10005094     MSVCRT:MSVCR120.dll
 0002:00000098       __imp____crtTerminateProcess 10005098     MSVCRT:MSVCR120.dll
 0002:0000009c       __imp_?terminate@@YAXXZ    1000509c     MSVCRT:MSVCR120.dll
 0002:000000a0       __imp____clean_type_info_names_internal 100050a0     MSVCRT:MSVCR120.dll
 0002:000000a4       __imp___amsg_exit          100050a4     MSVCRT:MSVCR120.dll
 0002:000000a8       \177MSVCR120_NULL_THUNK_DATA 100050a8     MSVCRT:MSVCR120.dll
 0002:000000ac       __imp_?dynamicMetaObject@QObjectData@@QBEPAUQMetaObject@@XZ 100050ac     Qt5Core:Qt5Core.dll
 0002:000000b0       __imp_?shared_null@QMapDataBase@@2U1@B 100050b0     Qt5Core:Qt5Core.dll
 0002:000000b4       __imp_?shared_null@QListData@@2UData@1@B 100050b4     Qt5Core:Qt5Core.dll
 0002:000000b8       __imp_?timerEvent@QObject@@MAEXPAVQTimerEvent@@@Z 100050b8     Qt5Core:Qt5Core.dll
 0002:000000bc       __imp_?eventFilter@QObject@@UAE_NPAV1@PAVQEvent@@@Z 100050bc     Qt5Core:Qt5Core.dll
 0002:000000c0       __imp_?event@QObject@@UAE_NPAVQEvent@@@Z 100050c0     Qt5Core:Qt5Core.dll
 0002:000000c4       __imp_?disconnectNotify@QObject@@MAEXABVQMetaMethod@@@Z 100050c4     Qt5Core:Qt5Core.dll
 0002:000000c8       __imp_?customEvent@QObject@@MAEXPAVQEvent@@@Z 100050c8     Qt5Core:Qt5Core.dll
 0002:000000cc       __imp_?connectNotify@QObject@@MAEXABVQMetaMethod@@@Z 100050cc     Qt5Core:Qt5Core.dll
 0002:000000d0       __imp_?childEvent@QObject@@MAEXPAVQChildEvent@@@Z 100050d0     Qt5Core:Qt5Core.dll
 0002:000000d4       __imp_??6QTextStream@@QAEAAV0@ABVQString@@@Z 100050d4     Qt5Core:Qt5Core.dll
 0002:000000d8       __imp_??1QTextStream@@UAE@XZ 100050d8     Qt5Core:Qt5Core.dll
 0002:000000dc       __imp_??0QTextStream@@QAE@PAVQIODevice@@@Z 100050dc     Qt5Core:Qt5Core.dll
 0002:000000e0       __imp_??1QVariant@@QAE@XZ  100050e0     Qt5Core:Qt5Core.dll
 0002:000000e4       __imp_?freeData@QMapDataBase@@SAXPAU1@@Z 100050e4     Qt5Core:Qt5Core.dll
 0002:000000e8       __imp_??0QString@@QAE@XZ   100050e8     Qt5Core:Qt5Core.dll
 0002:000000ec       __imp_??0QString@@QAE@PBVQChar@@H@Z 100050ec     Qt5Core:Qt5Core.dll
 0002:000000f0       __imp_??1QString@@QAE@XZ   100050f0     Qt5Core:Qt5Core.dll
 0002:000000f4       __imp_??4QString@@QAEAAV0@ABV0@@Z 100050f4     Qt5Core:Qt5Core.dll
 0002:000000f8       __imp_??4QString@@QAEAAV0@$$QAV0@@Z 100050f8     Qt5Core:Qt5Core.dll
 0002:000000fc       __imp_?data@QString@@QAEPAVQChar@@XZ 100050fc     Qt5Core:Qt5Core.dll
 0002:00000100       __imp_?indexOf@QString@@QBEHABV1@HW4CaseSensitivity@Qt@@@Z 10005100     Qt5Core:Qt5Core.dll
 0002:00000104       __imp_?left@QString@@QBE?AV1@H@Z 10005104     Qt5Core:Qt5Core.dll
 0002:00000108       __imp_?startsWith@QString@@QBE_NABV1@W4CaseSensitivity@Qt@@@Z 10005108     Qt5Core:Qt5Core.dll
 0002:0000010c       __imp_?trimmed@QString@@QBE?AV1@XZ 1000510c     Qt5Core:Qt5Core.dll
 0002:00000110       __imp_?simplified@QString@@QBE?AV1@XZ 10005110     Qt5Core:Qt5Core.dll
 0002:00000114       __imp_??8@YA_NABVQString@@0@Z 10005114     Qt5Core:Qt5Core.dll
 0002:00000118       __imp_?fromAscii_helper@QString@@CAPAU?$QTypedArrayData@G@@PBDH@Z 10005118     Qt5Core:Qt5Core.dll
 0002:0000011c       __imp_?tr@QMetaObject@@QBE?AVQString@@PBD0H@Z 1000511c     Qt5Core:Qt5Core.dll
 0002:00000120       __imp_??1Connection@QMetaObject@@QAE@XZ 10005120     Qt5Core:Qt5Core.dll
 0002:00000124       __imp_?detach_grow@QListData@@QAEPAUData@1@PAHH@Z 10005124     Qt5Core:Qt5Core.dll
 0002:00000128       __imp_?dispose@QListData@@SAXPAUData@1@@Z 10005128     Qt5Core:Qt5Core.dll
 0002:0000012c       __imp_?append@QListData@@QAEPAPAXXZ 1000512c     Qt5Core:Qt5Core.dll
 0002:00000130       __imp_?connect@QObject@@QBE?AVConnection@QMetaObject@@PBV1@PBD1W4ConnectionType@Qt@@@Z 10005130     Qt5Core:Qt5Core.dll
 0002:00000134       __imp_??0QFile@@QAE@ABVQString@@@Z 10005134     Qt5Core:Qt5Core.dll
 0002:00000138       __imp_??1QFile@@UAE@XZ     10005138     Qt5Core:Qt5Core.dll
 0002:0000013c       __imp_?open@QFile@@UAE_NV?$QFlags@W4OpenModeFlag@QIODevice@@@@@Z 1000513c     Qt5Core:Qt5Core.dll
 0002:00000140       __imp_?toNativeSeparators@QDir@@SA?AVQString@@ABV2@@Z 10005140     Qt5Core:Qt5Core.dll
 0002:00000144       __imp_?freeTree@QMapDataBase@@QAEXPAUQMapNodeBase@@H@Z 10005144     Qt5Core:Qt5Core.dll
 0002:00000148       \177Qt5Core_NULL_THUNK_DATA 10005148     Qt5Core:Qt5Core.dll
 0002:0000014c       __imp_?clipboard@QGuiApplication@@SAPAVQClipboard@@XZ 1000514c     Qt5Gui:Qt5Gui.dll
 0002:00000150       __imp_?setText@QClipboard@@QAEXABVQString@@W4Mode@1@@Z 10005150     Qt5Gui:Qt5Gui.dll
 0002:00000154       __imp_?text@QClipboard@@QBE?AVQString@@W4Mode@1@@Z 10005154     Qt5Gui:Qt5Gui.dll
 0002:00000158       \177Qt5Gui_NULL_THUNK_DATA 10005158     Qt5Gui:Qt5Gui.dll
 0002:0000015c       __imp_?getAppSettings@AppContext@U2@@SAPAVAppSettings@2@XZ 1000515c     U2Core:U2Core.dll
 0002:00000160       __imp_?getMainWindow@AppContext@U2@@SAPAVMainWindow@2@XZ 10005160     U2Core:U2Core.dll
 0002:00000164       __imp_?getTaskScheduler@AppContext@U2@@SAPAVTaskScheduler@2@XZ 10005164     U2Core:U2Core.dll
 0002:00000168       __imp_??0Logger@U2@@QAE@ABVQString@@@Z 10005168     U2Core:U2Core.dll
 0002:0000016c       __imp_??1Logger@U2@@UAE@XZ 1000516c     U2Core:U2Core.dll
 0002:00000170       __imp_??0GUrl@U2@@QAE@ABVQString@@W4GUrlType@1@@Z 10005170     U2Core:U2Core.dll
 0002:00000174       __imp_??0GUrl@U2@@QAE@ABV01@@Z 10005174     U2Core:U2Core.dll
 0002:00000178       __imp_??1GUrl@U2@@QAE@XZ   10005178     U2Core:U2Core.dll
 0002:0000017c       __imp_??1GCounter@U2@@UAE@XZ 1000517c     U2Core:U2Core.dll
 0002:00000180       __imp_?staticMetaObject@Plugin@U2@@2UQMetaObject@@B 10005180     U2Core:U2Core.dll
 0002:00000184       __imp_?qt_metacall@Plugin@U2@@UAEHW4Call@QMetaObject@@HPAPAX@Z 10005184     U2Core:U2Core.dll
 0002:00000188       __imp_?qt_metacast@Plugin@U2@@UAEPAXPBD@Z 10005188     U2Core:U2Core.dll
 0002:0000018c       __imp_??_7SimpleEventCounter@U2@@6B@ 1000518c     U2Core:U2Core.dll
 0002:00000190       __imp_?setReportingSupported@Task@U2@@UAEX_N@Z 10005190     U2Core:U2Core.dll
 0002:00000194       __imp_?setReportingEnabled@Task@U2@@UAEX_N@Z 10005194     U2Core:U2Core.dll
 0002:00000198       __imp_?setNotificationReport@Task@U2@@UAEX_N@Z 10005198     U2Core:U2Core.dll
 0002:0000019c       __imp_?setNoAutoDelete@Task@U2@@UAEX_N@Z 1000519c     U2Core:U2Core.dll
 0002:000001a0       __imp_?setCollectChildrensWarningsFlag@Task@U2@@UAEX_N@Z 100051a0     U2Core:U2Core.dll
 0002:000001a4       __imp_?run@Task@U2@@UAEXXZ 100051a4     U2Core:U2Core.dll
 0002:000001a8       __imp_?report@Task@U2@@UAE?AW4ReportResult@12@XZ 100051a8     U2Core:U2Core.dll
 0002:000001ac       __imp_?propagateSubtaskError@Task@U2@@UAE_NXZ 100051ac     U2Core:U2Core.dll
 0002:000001b0       __imp_?isTopLevelTask@Task@U2@@UBE_NXZ 100051b0     U2Core:U2Core.dll
 0002:000001b4       __imp_?isReportingSupported@Task@U2@@UBE_NXZ 100051b4     U2Core:U2Core.dll
 0002:000001b8       __imp_?isReportingEnabled@Task@U2@@UBE_NXZ 100051b8     U2Core:U2Core.dll
 0002:000001bc       __imp_?isNotificationReport@Task@U2@@UBE_NXZ 100051bc     U2Core:U2Core.dll
 0002:000001c0       __imp_?hasWarning@Task@U2@@UBE_NXZ 100051c0     U2Core:U2Core.dll
 0002:000001c4       __imp_?hasSubtasksWithErrors@Task@U2@@UBE_NXZ 100051c4     U2Core:U2Core.dll
 0002:000001c8       __imp_?getWarnings@Task@U2@@UBE?AVQStringList@@XZ 100051c8     U2Core:U2Core.dll
 0002:000001cc       __imp_?getTopLevelParentTask@Task@U2@@UAEPAV12@XZ 100051cc     U2Core:U2Core.dll
 0002:000001d0       __imp_?getTaskId@Task@U2@@UBE_JXZ 100051d0     U2Core:U2Core.dll
 0002:000001d4       __imp_?getSubtaskWithErrors@Task@U2@@UBEPAV12@XZ 100051d4     U2Core:U2Core.dll
 0002:000001d8       __imp_?getParentTask@Task@U2@@UBEPAV12@XZ 100051d8     U2Core:U2Core.dll
 0002:000001dc       __imp_?getNumParallelSubtasks@Task@U2@@UBEHXZ 100051dc     U2Core:U2Core.dll
 0002:000001e0       __imp_?cleanup@Task@U2@@UAEXXZ 100051e0     U2Core:U2Core.dll
 0002:000001e4       __imp_??1Plugin@U2@@UAE@XZ 100051e4     U2Core:U2Core.dll
 0002:000001e8       __imp_??0Plugin@U2@@QAE@ABVQString@@0_NW4PluginState@1@@Z 100051e8     U2Core:U2Core.dll
 0002:000001ec       __imp_?prepareTmpFileLocation@GUrlUtils@U2@@SA?AVQString@@ABV3@00AAVU2OpStatus@2@@Z 100051ec     U2Core:U2Core.dll
 0002:000001f0       __imp_??1U2OpStatus2Log@U2@@UAE@XZ 100051f0     U2Core:U2Core.dll
 0002:000001f4       __imp_??0U2OpStatus2Log@U2@@QAE@W4LogLevel@1@@Z 100051f4     U2Core:U2Core.dll
 0002:000001f8       __imp_?getDefaultDownloadDirectory@BaseLoadRemoteDocumentTask@U2@@SA?AVQString@@XZ 100051f8     U2Core:U2Core.dll
 0002:000001fc       __imp_?prepareDownloadDirectory@BaseLoadRemoteDocumentTask@U2@@SA_NAAVQString@@@Z 100051fc     U2Core:U2Core.dll
 0002:00000200       __imp_?getCurrentProcessTemporaryDirPath@UserAppsSettings@U2@@QBE?AVQString@@ABV3@@Z 10005200     U2Core:U2Core.dll
 0002:00000204       __imp_??1SimpleEventCounter@U2@@UAE@XZ 10005204     U2Core:U2Core.dll
 0002:00000208       __imp_??0GReportableCounter@U2@@QAE@ABVQString@@0N@Z 10005208     U2Core:U2Core.dll
 0002:0000020c       __imp_?getProjectLoader@AppContext@U2@@SAPAVProjectLoader@2@XZ 1000520c     U2Core:U2Core.dll
 0002:00000210       \177U2Core_NULL_THUNK_DATA 10005210     U2Core:U2Core.dll
 0002:00000214       __imp_??1LoadRemoteDocumentAndAddToProjectTask@U2@@UAE@XZ 10005214     U2Gui:U2Gui.dll
 0002:00000218       __imp_?generateReport@LoadRemoteDocumentAndAddToProjectTask@U2@@UBE?AVQString@@XZ 10005218     U2Gui:U2Gui.dll
 0002:0000021c       __imp_?metaObject@LoadRemoteDocumentAndAddToProjectTask@U2@@UBEPBUQMetaObject@@XZ 1000521c     U2Gui:U2Gui.dll
 0002:00000220       __imp_?onSubTaskFinished@LoadRemoteDocumentAndAddToProjectTask@U2@@MAE?AV?$QList@PAVTask@U2@@@@PAVTask@2@@Z 10005220     U2Gui:U2Gui.dll
 0002:00000224       __imp_?prepare@LoadRemoteDocumentAndAddToProjectTask@U2@@UAEXXZ 10005224     U2Gui:U2Gui.dll
 0002:00000228       __imp_?qt_metacall@LoadRemoteDocumentAndAddToProjectTask@U2@@UAEHW4Call@QMetaObject@@HPAPAX@Z 10005228     U2Gui:U2Gui.dll
 0002:0000022c       __imp_?qt_metacast@LoadRemoteDocumentAndAddToProjectTask@U2@@UAEPAXPBD@Z 1000522c     U2Gui:U2Gui.dll
 0002:00000230       __imp_??0LoadRemoteDocumentAndAddToProjectTask@U2@@QAE@ABVQString@@000ABV?$QMap@VQString@@VQVariant@@@@W4LoadRemoteDocumentMode@1@@Z 10005230     U2Gui:U2Gui.dll
 0002:00000234       \177U2Gui_NULL_THUNK_DATA  10005234     U2Gui:U2Gui.dll
 0002:00000238       ___xc_a                    10005238     MSVCRT:cinitexe.obj
 0002:00000274       ___xc_z                    10005274     MSVCRT:cinitexe.obj
 0002:00000278       ___xi_a                    10005278     MSVCRT:cinitexe.obj
 0002:00000284       ___xi_z                    10005284     MSVCRT:cinitexe.obj
 0002:000002c8       ??_C@_00CNPNBAHC@?$AA@     100052c8     BrowserSupportPlugin.obj
 0002:000002d0       ??_7error_category@std@@6B@ 100052d0     BrowserSupportPlugin.obj
 0002:000002ec       ??_7_Generic_error_category@std@@6B@ 100052ec     BrowserSupportPlugin.obj
 0002:00000304       ??_C@_07DCLBNMLN@generic?$AA@ 10005304     BrowserSupportPlugin.obj
 0002:0000030c       ??_C@_0O@BFJCFAAK@unknown?5error?$AA@ 1000530c     BrowserSupportPlugin.obj
 0002:00000320       ??_7_Iostream_error_category@std@@6B@ 10005320     BrowserSupportPlugin.obj
 0002:00000338       ??_C@_08LLGCOLLL@iostream?$AA@ 10005338     BrowserSupportPlugin.obj
 0002:00000344       ??_C@_0BG@PADBLCHM@iostream?5stream?5error?$AA@ 10005344     BrowserSupportPlugin.obj
 0002:00000360       ??_7_System_error_category@std@@6B@ 10005360     BrowserSupportPlugin.obj
 0002:00000378       ??_C@_06FHFOAHML@system?$AA@ 10005378     BrowserSupportPlugin.obj
 0002:00000380       ??_C@_0L@JLHNEGIN@Algorithms?$AA@ 10005380     BrowserSupportPlugin.obj
 0002:0000038c       ??_C@_07PGLPGHFC@Console?$AA@ 1000538c     BrowserSupportPlugin.obj
 0002:00000394       ??_C@_0O@BOFHOPCF@Core?5Services?$AA@ 10005394     BrowserSupportPlugin.obj
 0002:000003a4       ??_C@_0N@PPADAKBM@Input?1Output?$AA@ 100053a4     BrowserSupportPlugin.obj
 0002:000003b4       ??_C@_0M@KPPBKPKK@Performance?$AA@ 100053b4     BrowserSupportPlugin.obj
 0002:000003c0       ??_C@_07BFDHHBBI@Scripts?$AA@ 100053c0     BrowserSupportPlugin.obj
 0002:000003c8       ??_C@_05EEGKELMG@Tasks?$AA@ 100053c8     BrowserSupportPlugin.obj
 0002:000003d0       ??_C@_0P@NIIOBHGA@User?5Interface?$AA@ 100053d0     BrowserSupportPlugin.obj
 0002:000003e0       ??_C@_0N@JINCGGMN@User?5Actions?$AA@ 100053e0     BrowserSupportPlugin.obj
 0002:000003f4       ??_SLoadRemoteDocumentAndAddToProjectTask@U2@@6B@ 100053f4     BrowserSupportPlugin.obj
 0002:00000484       ??_7BrowserSupportPlugin@U2@@6B@ 10005484     BrowserSupportPlugin.obj
 0002:000004b0       ??_C@_0BA@BKIIJABN@Browser?5support?$AA@ 100054b0     BrowserSupportPlugin.obj
 0002:000004c0       ??_C@_0P@FODADHKH@BrowserSupport?$AA@ 100054c0     BrowserSupportPlugin.obj
 0002:000004d0       ??_C@_0BF@EFJCNFLL@1sl_clipboardCheck?$CI?$CJ?$AA@ 100054d0     BrowserSupportPlugin.obj
 0002:000004e8       ??_C@_0BL@BNKJLOEN@2changed?$CIQClipboard?3?3Mode?$CJ?$AA@ 100054e8     BrowserSupportPlugin.obj
 0002:00000504       ??_C@_09DEBOPNMH@clipboard?$AA@ 10005504     BrowserSupportPlugin.obj
 0002:00000510       ??_C@_0P@LPEFOGJP@clipboard_data?$AA@ 10005510     BrowserSupportPlugin.obj
 0002:00000520       ??_C@_01EEMJAFIK@?6?$AA@   10005520     BrowserSupportPlugin.obj
 0002:00000524       ??_C@_0BA@OFFODCOF@open?1selection?$DL?$AA@ 10005524     BrowserSupportPlugin.obj
 0002:00000534       ??_C@_0BO@FGGLEJEI@BrowserSupport?3open?1selection?$AA@ 10005534     BrowserSupportPlugin.obj
 0002:00000554       ??_C@_0O@BLNDMOIO@open?1Ensembl?$DL?$AA@ 10005554     BrowserSupportPlugin.obj
 0002:00000564       ??_C@_0BM@GLGLHBPF@BrowserSupport?3open?1Ensembl?$AA@ 10005564     BrowserSupportPlugin.obj
 0002:00000580       ??_C@_07LDDBJGBM@ENSEMBL?$AA@ 10005580     BrowserSupportPlugin.obj
 0002:00000588       ??_C@_09BKILJDBC@open?1PDB?$DL?$AA@ 10005588     BrowserSupportPlugin.obj
 0002:00000594       ??_C@_0BI@BHEBAGAE@BrowserSupport?3open?1PDB?$AA@ 10005594     BrowserSupportPlugin.obj
 0002:000005ac       ??_C@_03KAGKCHNK@PDB?$AA@  100055ac     BrowserSupportPlugin.obj
 0002:000005b0       ??_C@_0BA@JFNIOLAK@string?5too?5long?$AA@ 100055b0     BrowserSupportPlugin.obj
 0002:000005c0       ??_C@_0BI@CFPLBAOH@invalid?5string?5position?$AA@ 100055c0     BrowserSupportPlugin.obj
 0002:000005d8       __real@3ff0000000000000    100055d8     BrowserSupportPlugin.obj
 0002:00000694       ?value@?$integral_constant@_N$0A@@std@@2_NB 10005694     MSVCRT:ti_inst.obj
 0002:00000695       ?value@?$integral_constant@_N$00@std@@2_NB 10005695     MSVCRT:ti_inst.obj
 0002:0000069c       ??_7type_info@@6B@         1000569c     MSVCRT:ti_inst.obj
 0002:000006a0       __pRawDllMain              100056a0     MSVCRT:crtdll.obj
 0002:000006a0       __pDefaultRawDllMain       100056a0     MSVCRT:crtdll.obj
 0002:000006ac       ?ProcessDetach@NativeDll@<CrtImplementationDetails>@@0IB 100056ac     MSVCRT:initsect.obj
 0002:000006b0       ?ProcessAttach@NativeDll@<CrtImplementationDetails>@@0IB 100056b0     MSVCRT:initsect.obj
 0002:000006b4       ?ThreadAttach@NativeDll@<CrtImplementationDetails>@@0IB 100056b4     MSVCRT:initsect.obj
 0002:000006b8       ?ThreadDetach@NativeDll@<CrtImplementationDetails>@@0IB 100056b8     MSVCRT:initsect.obj
 0002:000006bc       ?ProcessVerifier@NativeDll@<CrtImplementationDetails>@@0IB 100056bc     MSVCRT:initsect.obj
 0002:000006c0       __load_config_used         100056c0     MSVCRT:loadcfg.obj
 0002:00000780       ??_R4error_category@std@@6B@ 10005780     BrowserSupportPlugin.obj
 0002:00000794       ??_R3error_category@std@@8 10005794     BrowserSupportPlugin.obj
 0002:000007a4       ??_R2error_category@std@@8 100057a4     BrowserSupportPlugin.obj
 0002:000007ac       ??_R1A@?0A@EA@error_category@std@@8 100057ac     BrowserSupportPlugin.obj
 0002:000007c8       ??_R4_Generic_error_category@std@@6B@ 100057c8     BrowserSupportPlugin.obj
 0002:000007dc       ??_R3_Generic_error_category@std@@8 100057dc     BrowserSupportPlugin.obj
 0002:000007ec       ??_R2_Generic_error_category@std@@8 100057ec     BrowserSupportPlugin.obj
 0002:000007f8       ??_R1A@?0A@EA@_Generic_error_category@std@@8 100057f8     BrowserSupportPlugin.obj
 0002:00000814       ??_R4_Iostream_error_category@std@@6B@ 10005814     BrowserSupportPlugin.obj
 0002:00000828       ??_R3_Iostream_error_category@std@@8 10005828     BrowserSupportPlugin.obj
 0002:00000838       ??_R2_Iostream_error_category@std@@8 10005838     BrowserSupportPlugin.obj
 0002:00000848       ??_R1A@?0A@EA@_Iostream_error_category@std@@8 10005848     BrowserSupportPlugin.obj
 0002:00000864       ??_R4_System_error_category@std@@6B@ 10005864     BrowserSupportPlugin.obj
 0002:00000878       ??_R3_System_error_category@std@@8 10005878     BrowserSupportPlugin.obj
 0002:00000888       ??_R2_System_error_category@std@@8 10005888     BrowserSupportPlugin.obj
 0002:00000898       ??_R1A@?0A@EA@_System_error_category@std@@8 10005898     BrowserSupportPlugin.obj
 0002:000008b4       ??_R1A@?0A@EA@QObject@@8   100058b4     BrowserSupportPlugin.obj
 0002:000008d0       ??_R3QObject@@8            100058d0     BrowserSupportPlugin.obj
 0002:000008e0       ??_R2QObject@@8            100058e0     BrowserSupportPlugin.obj
 0002:000008e8       ??_R4LoadRemoteDocumentAndAddToProjectTask@U2@@6B@ 100058e8     BrowserSupportPlugin.obj
 0002:000008fc       ??_R3LoadRemoteDocumentAndAddToProjectTask@U2@@8 100058fc     BrowserSupportPlugin.obj
 0002:0000090c       ??_R2LoadRemoteDocumentAndAddToProjectTask@U2@@8 1000590c     BrowserSupportPlugin.obj
 0002:0000091c       ??_R1A@?0A@EA@LoadRemoteDocumentAndAddToProjectTask@U2@@8 1000591c     BrowserSupportPlugin.obj
 0002:00000938       ??_R1A@?0A@EA@Task@U2@@8   10005938     BrowserSupportPlugin.obj
 0002:00000954       ??_R3Task@U2@@8            10005954     BrowserSupportPlugin.obj
 0002:00000964       ??_R2Task@U2@@8            10005964     BrowserSupportPlugin.obj
 0002:00000970       ??_R4BrowserSupportPlugin@U2@@6B@ 10005970     BrowserSupportPlugin.obj
 0002:00000984       ??_R3BrowserSupportPlugin@U2@@8 10005984     BrowserSupportPlugin.obj
 0002:00000994       ??_R2BrowserSupportPlugin@U2@@8 10005994     BrowserSupportPlugin.obj
 0002:000009a4       ??_R1A@?0A@EA@BrowserSupportPlugin@U2@@8 100059a4     BrowserSupportPlugin.obj
 0002:000009c0       ??_R1A@?0A@EA@Plugin@U2@@8 100059c0     BrowserSupportPlugin.obj
 0002:000009dc       ??_R3Plugin@U2@@8          100059dc     BrowserSupportPlugin.obj
 0002:000009ec       ??_R2Plugin@U2@@8          100059ec     BrowserSupportPlugin.obj
 0002:000009f8       ??_R4type_info@@6B@        100059f8     MSVCRT:ti_inst.obj
 0002:00000a0c       ??_R3type_info@@8          10005a0c     MSVCRT:ti_inst.obj
 0002:00000a1c       ??_R2type_info@@8          10005a1c     MSVCRT:ti_inst.obj
 0002:00000a24       ??_R1A@?0A@EA@type_info@@8 10005a24     MSVCRT:ti_inst.obj
 0002:00000a40       ___safe_se_handler_table   10005a40     <linker-defined>
 0002:00000a88       ___rtc_iaa                 10005a88     MSVCRT:initsect.obj
 0002:00000a8c       ___rtc_izz                 10005a8c     MSVCRT:initsect.obj
 0002:00000a90       ___rtc_taa                 10005a90     MSVCRT:initsect.obj
 0002:00000a94       ___rtc_tzz                 10005a94     MSVCRT:initsect.obj
 0002:00001208       __IMPORT_DESCRIPTOR_U2Core 10006208     U2Core:U2Core.dll
 0002:0000121c       __IMPORT_DESCRIPTOR_U2Gui  1000621c     U2Gui:U2Gui.dll
 0002:00001230       __IMPORT_DESCRIPTOR_Qt5Gui 10006230     Qt5Gui:Qt5Gui.dll
 0002:00001244       __IMPORT_DESCRIPTOR_Qt5Core 10006244     Qt5Core:Qt5Core.dll
 0002:00001258       __IMPORT_DESCRIPTOR_MSVCP120 10006258     msvcprt:MSVCP120.dll
 0002:0000126c       __IMPORT_DESCRIPTOR_MSVCR120 1000626c     MSVCRT:MSVCR120.dll
 0002:00001280       __IMPORT_DESCRIPTOR_KERNEL32 10006280     kernel32:KERNEL32.dll
 0002:00001294       __NULL_IMPORT_DESCRIPTOR   10006294     U2Core:U2Core.dll
 0003:00000000       ?_Generic_object@?$_Error_objects@H@std@@2V_Generic_error_category@2@A 10008000     BrowserSupportPlugin.obj
 0003:00000004       ?_Iostream_object@?$_Error_objects@H@std@@2V_Iostream_error_category@2@A 10008004     BrowserSupportPlugin.obj
 0003:00000008       ?_System_object@?$_Error_objects@H@std@@2V_System_error_category@2@A 10008008     BrowserSupportPlugin.obj
 0003:0000000c       ?staticMetaObject@BrowserSupportPlugin@U2@@2UQMetaObject@@B 1000800c     moc_BrowserSupportPlugin.obj
 0003:00000024       ___security_cookie         10008024     MSVCRT:gs_cookie.obj
 0003:00000028       ___security_cookie_complement 10008028     MSVCRT:gs_cookie.obj
 0003:00000030       ___native_dllmain_reason   10008030     MSVCRT:natstart.obj
 0003:00000034       ??_R0?AVerror_category@std@@@8 10008034     BrowserSupportPlugin.obj
 0003:00000058       ??_R0?AV_Generic_error_category@std@@@8 10008058     BrowserSupportPlugin.obj
 0003:00000084       ??_R0?AV_Iostream_error_category@std@@@8 10008084     BrowserSupportPlugin.obj
 0003:000000b0       ??_R0?AV_System_error_category@std@@@8 100080b0     BrowserSupportPlugin.obj
 0003:000000dc       ??_R0?AVQObject@@@8        100080dc     BrowserSupportPlugin.obj
 0003:000000f4       ??_R0?AVLoadRemoteDocumentAndAddToProjectTask@U2@@@8 100080f4     BrowserSupportPlugin.obj
 0003:0000012c       ??_R0?AVTask@U2@@@8        1000812c     BrowserSupportPlugin.obj
 0003:00000144       ??_R0?AVBrowserSupportPlugin@U2@@@8 10008144     BrowserSupportPlugin.obj
 0003:0000016c       ??_R0?AVPlugin@U2@@@8      1000816c     BrowserSupportPlugin.obj
 0003:00000184       ??_R0?AVtype_info@@@8      10008184     MSVCRT:ti_inst.obj
 0003:000001f0       ?id@?$num_put@DV?$back_insert_iterator@V?$basic_string@DU?$char_traits@D@std@@V?$allocator@D@2@@std@@@std@@@std@@2V0locale@2@A 100081f0     BrowserSupportPlugin.obj
 0003:000001f4       ?id@?$num_put@_WV?$back_insert_iterator@V?$basic_string@_WU?$char_traits@_W@std@@V?$allocator@_W@2@@std@@@std@@@std@@2V0locale@2@A 100081f4     BrowserSupportPlugin.obj
 0003:000005a0       ?__type_info_root_node@@3U__type_info_node@@A 100085a0     MSVCRT:tncleanup.obj
 0003:000005a8       ___native_startup_lock     100085a8     <common>
 0003:000005ac       ___native_startup_state    100085ac     <common>
 0003:000005b0       ___dyn_tls_init_callback   100085b0     <common>
 0003:000005b4       ___onexitend               100085b4     <common>
 0003:000005b8       ___onexitbegin             100085b8     <common>

 entry point at        0001:00002d2a

 Static symbols

 0000:ffff5000       .debug$S                   10000000     MSVCRT:MSVCR120.dll
 0000:ffff5000       .debug$S                   10000000     MSVCRT:MSVCR120.dll
 0000:ffff5000       .debug$S                   10000000     MSVCRT:MSVCR120.dll
 0000:ffff5000       .debug$S                   10000000     MSVCRT:MSVCR120.dll
 0000:ffff5000       .debug$S                   10000000     MSVCRT:MSVCR120.dll
 0000:ffff5000       .debug$S                   10000000     MSVCRT:MSVCR120.dll
 0000:ffff5000       .debug$S                   10000000     MSVCRT:MSVCR120.dll
 0000:ffff5000       .debug$S                   10000000     msvcprt:MSVCP120.dll
 0000:ffff5000       .debug$S                   10000000     msvcprt:MSVCP120.dll
 0000:ffff5000       .debug$S                   10000000     kernel32:KERNEL32.dll
 0000:ffff5000       .debug$S                   10000000     kernel32:KERNEL32.dll
 0000:ffff5000       .debug$S                   10000000     kernel32:KERNEL32.dll
 0000:ffff5000       .debug$S                   10000000     kernel32:KERNEL32.dll
 0000:ffff5000       .debug$S                   10000000     kernel32:KERNEL32.dll
 0000:ffff5000       .debug$S                   10000000     kernel32:KERNEL32.dll
 0000:ffff5000       .debug$S                   10000000     kernel32:KERNEL32.dll
 0001:fffff000       __ehhandler$?_Copy@?$basic_string@DU?$char_traits@D@std@@V?$allocator@D@2@@std@@QAEXII@Z 10000000 f   moc_BrowserSupportPlugin.obj
 0000:ffff5000       .debug$S                   10000000     kernel32:KERNEL32.dll
 0000:ffff5000       .debug$S                   10000000     kernel32:KERNEL32.dll
 0000:ffff5000       .debug$S                   10000000     msvcprt:MSVCP120.dll
 0000:ffff5000       .debug$S                   10000000     Qt5Core:Qt5Core.dll
 0000:ffff5000       .debug$S                   10000000     Qt5Core:Qt5Core.dll
 0000:ffff5000       .debug$S                   10000000     Qt5Core:Qt5Core.dll
 0002:ffffb000       __catchsym$?_Copy@?$basic_string@DU?$char_traits@D@std@@V?$allocator@D@2@@std@@QAEXII@Z$5 10000000     moc_BrowserSupportPlugin.obj
 0000:ffff5000       .debug$S                   10000000     MSVCRT:MSVCR120.dll
 0000:ffff5000       .debug$S                   10000000     MSVCRT:MSVCR120.dll
 0000:ffff5000       .debug$S                   10000000     MSVCRT:MSVCR120.dll
 0000:ffff5000       .debug$S                   10000000     MSVCRT:MSVCR120.dll
 0000:ffff5000       .debug$S                   10000000     Qt5Core:Qt5Core.dll
 0002:ffffb000       ?_Generic_object$initializer$@?$_Error_objects@H@std@@2P6AXXZA 10000000     moc_BrowserSupportPlugin.obj
 0002:ffffb000       ?_Iostream_object$initializer$@?$_Error_objects@H@std@@2P6AXXZA 10000000     moc_BrowserSupportPlugin.obj
 0002:ffffb000       ?_System_object$initializer$@?$_Error_objects@H@std@@2P6AXXZA 10000000     moc_BrowserSupportPlugin.obj
 0000:ffff5000       .debug$S                   10000000     Qt5Core:Qt5Core.dll
 0000:ffff5000       .debug$S                   10000000     Qt5Core:Qt5Core.dll
 0000:ffff5000       .debug$S                   10000000     Qt5Core:Qt5Core.dll
 0000:ffff5000       .debug$S                   10000000     Qt5Core:Qt5Core.dll
 0000:ffff5000       .debug$S                   10000000     Qt5Core:Qt5Core.dll
 0000:ffff5000       .debug$S                   10000000     Qt5Core:Qt5Core.dll
 0000:ffff5000       .debug$S                   10000000     Qt5Core:Qt5Core.dll
 0000:ffff5000       .debug$S                   10000000     Qt5Core:Qt5Core.dll
 0000:ffff5000       .debug$S                   10000000     Qt5Core:Qt5Core.dll
 0000:ffff5000       .debug$S                   10000000     Qt5Core:Qt5Core.dll
 0000:ffff5000       .debug$S                   10000000     Qt5Core:Qt5Core.dll
 0000:ffff5000       .debug$S                   10000000     Qt5Core:Qt5Core.dll
 0000:ffff5000       .debug$S                   10000000     Qt5Core:Qt5Core.dll
 0000:ffff5000       .debug$S                   10000000     Qt5Core:Qt5Core.dll
 0000:ffff5000       .debug$S                   10000000     Qt5Core:Qt5Core.dll
 0000:ffff5000       .debug$S                   10000000     Qt5Core:Qt5Core.dll
 0000:ffff5000       .debug$S                   10000000     Qt5Core:Qt5Core.dll
 0000:ffff5000       .debug$S                   10000000     Qt5Core:Qt5Core.dll
 0000:ffff5000       .debug$S                   10000000     Qt5Core:Qt5Core.dll
 0000:ffff5000       .debug$S                   10000000     Qt5Core:Qt5Core.dll
 0000:ffff5000       .debug$S                   10000000     Qt5Core:Qt5Core.dll
 0000:ffff5000       .debug$S                   10000000     Qt5Core:Qt5Core.dll
 0000:ffff5000       .debug$S                   10000000     Qt5Core:Qt5Core.dll
 0000:ffff5000       .debug$S                   10000000     Qt5Core:Qt5Core.dll
 0000:ffff5000       .debug$S                   10000000     Qt5Core:Qt5Core.dll
 0000:ffff5000       .debug$S                   10000000     Qt5Core:Qt5Core.dll
 0000:ffff5000       .debug$S                   10000000     Qt5Core:Qt5Core.dll
 0000:ffff5000       .debug$S                   10000000     Qt5Core:Qt5Core.dll
 0000:ffff5000       .debug$S                   10000000     Qt5Core:Qt5Core.dll
 0000:ffff5000       .debug$S                   10000000     Qt5Core:Qt5Core.dll
 0000:ffff5000       .debug$S                   10000000     Qt5Core:Qt5Core.dll
 0000:ffff5000       .debug$S                   10000000     Qt5Core:Qt5Core.dll
 0000:ffff5000       .debug$S                   10000000     Qt5Core:Qt5Core.dll
 0000:ffff5000       .debug$S                   10000000     Qt5Core:Qt5Core.dll
 0000:ffff5000       .debug$S                   10000000     Qt5Core:Qt5Core.dll
 0000:ffff5000       .debug$S                   10000000     msvcprt:MSVCP120.dll
 0000:ffff5000       .debug$S                   10000000     Qt5Gui:Qt5Gui.dll
 0000:ffff5000       .debug$S                   10000000     Qt5Gui:Qt5Gui.dll
 0000:ffff5000       .debug$S                   10000000     Qt5Gui:Qt5Gui.dll
 0000:ffff5000       .debug$S                   10000000     U2Gui:U2Gui.dll
 0000:ffff5000       .debug$S                   10000000     U2Gui:U2Gui.dll
 0000:ffff5000       .debug$S                   10000000     U2Gui:U2Gui.dll
 0000:ffff5000       .debug$S                   10000000     U2Gui:U2Gui.dll
 0000:ffff5000       .debug$S                   10000000     U2Gui:U2Gui.dll
 0000:ffff5000       .debug$S                   10000000     U2Gui:U2Gui.dll
 0000:ffff5000       .debug$S                   10000000     U2Gui:U2Gui.dll
 0000:ffff5000       .debug$S                   10000000     U2Gui:U2Gui.dll
 0000:ffff5000       .debug$S                   10000000     U2Core:U2Core.dll
 0000:ffff5000       .debug$S                   10000000     U2Core:U2Core.dll
 0000:ffff5000       .debug$S                   10000000     U2Core:U2Core.dll
 0000:ffff5000       .debug$S                   10000000     U2Core:U2Core.dll
 0000:ffff5000       .debug$S                   10000000     U2Core:U2Core.dll
 0000:ffff5000       .debug$S                   10000000     U2Core:U2Core.dll
 0000:ffff5000       .debug$S                   10000000     U2Core:U2Core.dll
 0000:ffff5000       .debug$S                   10000000     U2Core:U2Core.dll
 0000:ffff5000       .debug$S                   10000000     U2Core:U2Core.dll
 0000:ffff5000       .debug$S                   10000000     U2Core:U2Core.dll
 0000:ffff5000       .debug$S                   10000000     U2Core:U2Core.dll
 0000:ffff5000       .debug$S                   10000000     U2Core:U2Core.dll
 0000:ffff5000       .debug$S                   10000000     U2Core:U2Core.dll
 0000:ffff5000       .debug$S                   10000000     U2Core:U2Core.dll
 0000:ffff5000       .debug$S                   10000000     U2Core:U2Core.dll
 0000:ffff5000       .debug$S                   10000000     U2Core:U2Core.dll
 0000:ffff5000       .debug$S                   10000000     U2Core:U2Core.dll
 0000:ffff5000       .debug$S                   10000000     U2Core:U2Core.dll
 0000:ffff5000       .debug$S                   10000000     U2Core:U2Core.dll
 0000:ffff5000       .debug$S                   10000000     U2Core:U2Core.dll
 0000:ffff5000       .debug$S                   10000000     U2Core:U2Core.dll
 0000:ffff5000       .debug$S                   10000000     U2Core:U2Core.dll
 0000:ffff5000       .debug$S                   10000000     U2Core:U2Core.dll
 0000:ffff5000       .debug$S                   10000000     U2Core:U2Core.dll
 0000:ffff5000       .debug$S                   10000000     U2Core:U2Core.dll
 0000:ffff5000       .debug$S                   10000000     U2Core:U2Core.dll
 0000:ffff5000       .debug$S                   10000000     U2Core:U2Core.dll
 0000:ffff5000       .debug$S                   10000000     U2Core:U2Core.dll
 0000:ffff5000       .debug$S                   10000000     U2Core:U2Core.dll
 0000:ffff5000       .debug$S                   10000000     U2Core:U2Core.dll
 0000:ffff5000       .debug$S                   10000000     U2Core:U2Core.dll
 0000:ffff5000       .debug$S                   10000000     U2Core:U2Core.dll
 0000:ffff5000       .debug$S                   10000000     U2Core:U2Core.dll
 0000:ffff5000       .debug$S                   10000000     U2Core:U2Core.dll
 0000:ffff5000       .debug$S                   10000000     U2Core:U2Core.dll
 0000:ffff5000       .debug$S                   10000000     U2Core:U2Core.dll
 0000:ffff5000       .debug$S                   10000000     U2Core:U2Core.dll
 0000:ffff5000       .debug$S                   10000000     U2Core:U2Core.dll
 0000:ffff5000       .debug$S                   10000000     U2Core:U2Core.dll
 0000:ffff5000       .debug$S                   10000000     U2Core:U2Core.dll
 0000:ffff5000       .debug$S                   10000000     U2Core:U2Core.dll
 0000:ffff5000       .debug$S                   10000000     U2Core:U2Core.dll
 0000:ffff5000       .debug$S                   10000000     U2Core:U2Core.dll
 0000:ffff5000       .debug$S                   10000000     U2Core:U2Core.dll
 0000:ffff5000       .debug$S                   10000000     U2Core:U2Core.dll
 0000:ffff5000       .debug$S                   10000000     MSVCRT:MSVCR120.dll
 0000:ffff5000       .debug$S                   10000000     MSVCRT:MSVCR120.dll
 0000:ffff5000       .debug$S                   10000000     MSVCRT:MSVCR120.dll
 0000:ffff5000       .debug$S                   10000000     MSVCRT:MSVCR120.dll
 0000:ffff5000       .debug$S                   10000000     MSVCRT:MSVCR120.dll
 0000:ffff5000       .debug$S                   10000000     MSVCRT:MSVCR120.dll
 0000:ffff5000       .debug$S                   10000000     MSVCRT:MSVCR120.dll
 0000:ffff5000       .debug$S                   10000000     MSVCRT:MSVCR120.dll
 0000:ffff5000       .debug$S                   10000000     MSVCRT:MSVCR120.dll
 0000:ffff5000       .debug$S                   10000000     MSVCRT:MSVCR120.dll
 0000:ffff5000       .debug$S                   10000000     MSVCRT:MSVCR120.dll
 0000:ffff5000       .debug$S                   10000000     MSVCRT:MSVCR120.dll
 0000:ffff5000       .debug$S                   10000000     MSVCRT:MSVCR120.dll
 0000:ffff5000       .debug$S                   10000000     MSVCRT:MSVCR120.dll
 0000:ffff5000       .debug$S                   10000000     MSVCRT:MSVCR120.dll
 0000:ffff5000       .debug$S                   10000000     msvcprt:MSVCP120.dll
 0002:ffffb010       __catchsym$?_Copy@?$basic_string@DU?$char_traits@D@std@@V?$allocator@D@2@@std@@QAEXII@Z$4 10000010     moc_BrowserSupportPlugin.obj
 0002:ffffb020       __unwindtable$?_Copy@?$basic_string@DU?$char_traits@D@std@@V?$allocator@D@2@@std@@QAEXII@Z 10000020     moc_BrowserSupportPlugin.obj
 0002:ffffb040       __ehfuncinfo$?_Copy@?$basic_string@DU?$char_traits@D@std@@V?$allocator@D@2@@std@@QAEXII@Z 10000040     moc_BrowserSupportPlugin.obj
 0002:ffffb064       __tryblocktable$?_Copy@?$basic_string@DU?$char_traits@D@std@@V?$allocator@D@2@@std@@QAEXII@Z 10000064     moc_BrowserSupportPlugin.obj
 0001:fffff096       __catch$?_Copy@?$basic_string@DU?$char_traits@D@std@@V?$allocator@D@2@@std@@QAEXII@Z$0 10000096 f   moc_BrowserSupportPlugin.obj
 0001:fffff0d3       __catch$?_Copy@?$basic_string@DU?$char_traits@D@std@@V?$allocator@D@2@@std@@QAEXII@Z$1 100000d3 f   moc_BrowserSupportPlugin.obj
 0001:00000000       ??__E?_Generic_object@?$_Error_objects@H@std@@2V_Generic_error_category@2@A@@YAXXZ 10001000 f   BrowserSupportPlugin.obj
 0001:00000010       ??__E?_Iostream_object@?$_Error_objects@H@std@@2V_Iostream_error_category@2@A@@YAXXZ 10001010 f   BrowserSupportPlugin.obj
 0001:00000020       ??__E?_System_object@?$_Error_objects@H@std@@2V_System_error_category@2@A@@YAXXZ 10001020 f   BrowserSupportPlugin.obj
 0001:00000030       ??__EalgoLog@U2@@YAXXZ     10001030 f   BrowserSupportPlugin.obj
 0001:000000b0       ??__EcmdLog@U2@@YAXXZ      100010b0 f   BrowserSupportPlugin.obj
 0001:00000130       ??__EcoreLog@U2@@YAXXZ     10001130 f   BrowserSupportPlugin.obj
 0001:000001b0       ??__EioLog@U2@@YAXXZ       100011b0 f   BrowserSupportPlugin.obj
 0001:00000230       ??__EperfLog@U2@@YAXXZ     10001230 f   BrowserSupportPlugin.obj
 0001:000002b0       ??__EprevClipboard@U2@@YAXXZ 100012b0 f   BrowserSupportPlugin.obj
 0001:000002d0       ??__EscriptLog@U2@@YAXXZ   100012d0 f   BrowserSupportPlugin.obj
 0001:00000350       ??__EtaskLog@U2@@YAXXZ     10001350 f   BrowserSupportPlugin.obj
 0001:000003d0       ??__EuiLog@U2@@YAXXZ       100013d0 f   BrowserSupportPlugin.obj
 0001:00000450       ??__EuserActLog@U2@@YAXXZ  10001450 f   BrowserSupportPlugin.obj
 0001:000004d0       ??__E?_Generic_object@?$_Error_objects@H@std@@2V_Generic_error_category@2@A@@YAXXZ 100014d0 f   moc_BrowserSupportPlugin.obj
 0001:000004e0       ??__E?_Iostream_object@?$_Error_objects@H@std@@2V_Iostream_error_category@2@A@@YAXXZ 100014e0 f   moc_BrowserSupportPlugin.obj
 0001:000004f0       ??__E?_System_object@?$_Error_objects@H@std@@2V_System_error_category@2@A@@YAXXZ 100014f0 f   moc_BrowserSupportPlugin.obj
 0001:00000500       ??__E?staticMetaObject@BrowserSupportPlugin@U2@@2UQMetaObject@@B@@YAXXZ 10001500 f   moc_BrowserSupportPlugin.obj
 0001:00000c96       __catch$?_Copy@?$basic_string@DU?$char_traits@D@std@@V?$allocator@D@2@@std@@QAEXII@Z$0 10001c96 f i BrowserSupportPlugin.obj
 0001:00000cd3       __catch$?_Copy@?$basic_string@DU?$char_traits@D@std@@V?$allocator@D@2@@std@@QAEXII@Z$1 10001cd3 f i BrowserSupportPlugin.obj
 0001:00001010       __catch$?append@?$QList@VGUrl@U2@@@@QAEXABVGUrl@U2@@@Z$2 10002010 f i BrowserSupportPlugin.obj
 0001:00001010       __catch$?append@?$QList@VGUrl@U2@@@@QAEXABVGUrl@U2@@@Z$0 10002010 f i BrowserSupportPlugin.obj
 0001:0000158f       __catch$?detach_helper_grow@?$QList@VGUrl@U2@@@@AAEPAUNode@1@HH@Z$2 1000258f f i BrowserSupportPlugin.obj
 0001:000015ca       __catch$?detach_helper_grow@?$QList@VGUrl@U2@@@@AAEPAUNode@1@HH@Z$0 100025ca f i BrowserSupportPlugin.obj
 0001:00001a7e       __catch$?node_copy@?$QList@VGUrl@U2@@@@AAEXPAUNode@1@00@Z$0 10002a7e f i BrowserSupportPlugin.obj
 0001:00002ae0       _pre_c_init                10003ae0 f   MSVCRT:crtdll.obj
 0001:00002d4d       ___DllMainCRTStartup       10003d4d f   MSVCRT:crtdll.obj
 0001:00002ea0       $$000000                   10003ea0     MSVCRT:sehprolg4.obj
 0001:000032b5       ?ArrayUnwindFilter@@YAHPAU_EXCEPTION_POINTERS@@@Z 100042b5 f   MSVCRT:ehvecdtr.obj
 0001:00003600       __unwindfunclet$??0BrowserSupportPlugin@U2@@QAE@XZ$0 10004600 f   BrowserSupportPlugin.obj
 0001:00003609       __unwindfunclet$??0BrowserSupportPlugin@U2@@QAE@XZ$1 10004609 f   BrowserSupportPlugin.obj
 0001:00003612       __unwindfunclet$??0BrowserSupportPlugin@U2@@QAE@XZ$2 10004612 f   BrowserSupportPlugin.obj
 0001:0000361b       __ehhandler$??0BrowserSupportPlugin@U2@@QAE@XZ 1000461b f   BrowserSupportPlugin.obj
 0001:00003640       __unwindfunclet$??__EalgoLog@U2@@YAXXZ$0 10004640 f   BrowserSupportPlugin.obj
 0001:00003649       __ehhandler$??__EalgoLog@U2@@YAXXZ 10004649 f   BrowserSupportPlugin.obj
 0001:00003670       __unwindfunclet$??__EcmdLog@U2@@YAXXZ$0 10004670 f   BrowserSupportPlugin.obj
 0001:00003679       __ehhandler$??__EcmdLog@U2@@YAXXZ 10004679 f   BrowserSupportPlugin.obj
 0001:000036a0       __unwindfunclet$??__EcoreLog@U2@@YAXXZ$0 100046a0 f   BrowserSupportPlugin.obj
 0001:000036a9       __ehhandler$??__EcoreLog@U2@@YAXXZ 100046a9 f   BrowserSupportPlugin.obj
 0001:000036d0       __unwindfunclet$??__EioLog@U2@@YAXXZ$0 100046d0 f   BrowserSupportPlugin.obj
 0001:000036d9       __ehhandler$??__EioLog@U2@@YAXXZ 100046d9 f   BrowserSupportPlugin.obj
 0001:00003700       __unwindfunclet$??__EperfLog@U2@@YAXXZ$0 10004700 f   BrowserSupportPlugin.obj
 0001:00003709       __ehhandler$??__EperfLog@U2@@YAXXZ 10004709 f   BrowserSupportPlugin.obj
 0001:00003730       __unwindfunclet$??__EscriptLog@U2@@YAXXZ$0 10004730 f   BrowserSupportPlugin.obj
 0001:00003739       __ehhandler$??__EscriptLog@U2@@YAXXZ 10004739 f   BrowserSupportPlugin.obj
 0001:00003760       __unwindfunclet$??__EtaskLog@U2@@YAXXZ$0 10004760 f   BrowserSupportPlugin.obj
 0001:00003769       __ehhandler$??__EtaskLog@U2@@YAXXZ 10004769 f   BrowserSupportPlugin.obj
 0001:00003790       __unwindfunclet$??__EuiLog@U2@@YAXXZ$0 10004790 f   BrowserSupportPlugin.obj
 0001:00003799       __ehhandler$??__EuiLog@U2@@YAXXZ 10004799 f   BrowserSupportPlugin.obj
 0001:000037c0       __unwindfunclet$??__EuserActLog@U2@@YAXXZ$0 100047c0 f   BrowserSupportPlugin.obj
 0001:000037c9       __ehhandler$??__EuserActLog@U2@@YAXXZ 100047c9 f   BrowserSupportPlugin.obj
 0001:000037f0       __ehhandler$?_Copy@?$basic_string@DU?$char_traits@D@std@@V?$allocator@D@2@@std@@QAEXII@Z 100047f0 f   BrowserSupportPlugin.obj
 0001:00003810       __unwindfunclet$?append@?$QList@VGUrl@U2@@@@QAEXABVGUrl@U2@@@Z$6 10004810 f   BrowserSupportPlugin.obj
 0001:0000381b       __ehhandler$?append@?$QList@VGUrl@U2@@@@QAEXABVGUrl@U2@@@Z 1000481b f   BrowserSupportPlugin.obj
 0001:00003840       __ehhandler$?detach_helper_grow@?$QList@VGUrl@U2@@@@AAEPAUNode@1@HH@Z 10004840 f   BrowserSupportPlugin.obj
 0001:00003860       __unwindfunclet$?node_construct@?$QList@VGUrl@U2@@@@AAEXPAUNode@1@ABVGUrl@U2@@@Z$0 10004860 f   BrowserSupportPlugin.obj
 0001:0000386b       __ehhandler$?node_construct@?$QList@VGUrl@U2@@@@AAEXPAUNode@1@ABVGUrl@U2@@@Z 1000486b f   BrowserSupportPlugin.obj
 0001:00003890       __unwindfunclet$?node_copy@?$QList@VGUrl@U2@@@@AAEXPAUNode@1@00@Z$4 10004890 f   BrowserSupportPlugin.obj
 0001:0000389b       __ehhandler$?node_copy@?$QList@VGUrl@U2@@@@AAEXPAUNode@1@00@Z 1000489b f   BrowserSupportPlugin.obj
 0001:000038c0       __unwindfunclet$?saveToTmp@BrowserSupportPlugin@U2@@IAE?AVQString@@AAV3@@Z$0 100048c0 f   BrowserSupportPlugin.obj
 0001:000038c9       __unwindfunclet$?saveToTmp@BrowserSupportPlugin@U2@@IAE?AVQString@@AAV3@@Z$1 100048c9 f   BrowserSupportPlugin.obj
 0001:000038d2       __unwindfunclet$?saveToTmp@BrowserSupportPlugin@U2@@IAE?AVQString@@AAV3@@Z$2 100048d2 f   BrowserSupportPlugin.obj
 0001:000038db       __unwindfunclet$?saveToTmp@BrowserSupportPlugin@U2@@IAE?AVQString@@AAV3@@Z$3 100048db f   BrowserSupportPlugin.obj
 0001:000038e4       __unwindfunclet$?saveToTmp@BrowserSupportPlugin@U2@@IAE?AVQString@@AAV3@@Z$4 100048e4 f   BrowserSupportPlugin.obj
 0001:000038ed       __unwindfunclet$?saveToTmp@BrowserSupportPlugin@U2@@IAE?AVQString@@AAV3@@Z$5 100048ed f   BrowserSupportPlugin.obj
 0001:00003907       __unwindfunclet$?saveToTmp@BrowserSupportPlugin@U2@@IAE?AVQString@@AAV3@@Z$6 10004907 f   BrowserSupportPlugin.obj
 0001:00003910       __unwindfunclet$?saveToTmp@BrowserSupportPlugin@U2@@IAE?AVQString@@AAV3@@Z$7 10004910 f   BrowserSupportPlugin.obj
 0001:00003919       __ehhandler$?saveToTmp@BrowserSupportPlugin@U2@@IAE?AVQString@@AAV3@@Z 10004919 f   BrowserSupportPlugin.obj
 0001:00003940       __unwindfunclet$?sl_clipboardCheck@BrowserSupportPlugin@U2@@IAEXXZ$0 10004940 f   BrowserSupportPlugin.obj
 0001:00003949       __unwindfunclet$?sl_clipboardCheck@BrowserSupportPlugin@U2@@IAEXXZ$1 10004949 f   BrowserSupportPlugin.obj
 0001:00003952       __unwindfunclet$?sl_clipboardCheck@BrowserSupportPlugin@U2@@IAEXXZ$2 10004952 f   BrowserSupportPlugin.obj
 0001:0000395b       __unwindfunclet$?sl_clipboardCheck@BrowserSupportPlugin@U2@@IAEXXZ$3 1000495b f   BrowserSupportPlugin.obj
 0001:00003964       __unwindfunclet$?sl_clipboardCheck@BrowserSupportPlugin@U2@@IAEXXZ$4 10004964 f   BrowserSupportPlugin.obj
 0001:0000396d       __unwindfunclet$?sl_clipboardCheck@BrowserSupportPlugin@U2@@IAEXXZ$5 1000496d f   BrowserSupportPlugin.obj
 0001:0000397b       __unwindfunclet$?sl_clipboardCheck@BrowserSupportPlugin@U2@@IAEXXZ$6 1000497b f   BrowserSupportPlugin.obj
 0001:00003984       __unwindfunclet$?sl_clipboardCheck@BrowserSupportPlugin@U2@@IAEXXZ$7 10004984 f   BrowserSupportPlugin.obj
 0001:0000398d       __unwindfunclet$?sl_clipboardCheck@BrowserSupportPlugin@U2@@IAEXXZ$8 1000498d f   BrowserSupportPlugin.obj
 0001:00003996       __unwindfunclet$?sl_clipboardCheck@BrowserSupportPlugin@U2@@IAEXXZ$9 10004996 f   BrowserSupportPlugin.obj
 0001:0000399f       __unwindfunclet$?sl_clipboardCheck@BrowserSupportPlugin@U2@@IAEXXZ$10 1000499f f   BrowserSupportPlugin.obj
 0001:000039a7       __unwindfunclet$?sl_clipboardCheck@BrowserSupportPlugin@U2@@IAEXXZ$11 100049a7 f   BrowserSupportPlugin.obj
 0001:000039b0       __unwindfunclet$?sl_clipboardCheck@BrowserSupportPlugin@U2@@IAEXXZ$12 100049b0 f   BrowserSupportPlugin.obj
 0001:000039b8       __unwindfunclet$?sl_clipboardCheck@BrowserSupportPlugin@U2@@IAEXXZ$13 100049b8 f   BrowserSupportPlugin.obj
 0001:000039c1       __unwindfunclet$?sl_clipboardCheck@BrowserSupportPlugin@U2@@IAEXXZ$14 100049c1 f   BrowserSupportPlugin.obj
 0001:000039ca       __unwindfunclet$?sl_clipboardCheck@BrowserSupportPlugin@U2@@IAEXXZ$15 100049ca f   BrowserSupportPlugin.obj
 0001:000039d3       __unwindfunclet$?sl_clipboardCheck@BrowserSupportPlugin@U2@@IAEXXZ$16 100049d3 f   BrowserSupportPlugin.obj
 0001:000039dc       __unwindfunclet$?sl_clipboardCheck@BrowserSupportPlugin@U2@@IAEXXZ$17 100049dc f   BrowserSupportPlugin.obj
 0001:000039ea       __unwindfunclet$?sl_clipboardCheck@BrowserSupportPlugin@U2@@IAEXXZ$18 100049ea f   BrowserSupportPlugin.obj
 0001:000039f3       __unwindfunclet$?sl_clipboardCheck@BrowserSupportPlugin@U2@@IAEXXZ$19 100049f3 f   BrowserSupportPlugin.obj
 0001:000039fc       __unwindfunclet$?sl_clipboardCheck@BrowserSupportPlugin@U2@@IAEXXZ$20 100049fc f   BrowserSupportPlugin.obj
 0001:00003a05       __unwindfunclet$?sl_clipboardCheck@BrowserSupportPlugin@U2@@IAEXXZ$21 10004a05 f   BrowserSupportPlugin.obj
 0001:00003a0e       __unwindfunclet$?sl_clipboardCheck@BrowserSupportPlugin@U2@@IAEXXZ$22 10004a0e f   BrowserSupportPlugin.obj
 0001:00003a17       __unwindfunclet$?sl_clipboardCheck@BrowserSupportPlugin@U2@@IAEXXZ$23 10004a17 f   BrowserSupportPlugin.obj
 0001:00003a20       __unwindfunclet$?sl_clipboardCheck@BrowserSupportPlugin@U2@@IAEXXZ$24 10004a20 f   BrowserSupportPlugin.obj
 0001:00003a2b       __unwindfunclet$?sl_clipboardCheck@BrowserSupportPlugin@U2@@IAEXXZ$25 10004a2b f   BrowserSupportPlugin.obj
 0001:00003a45       __unwindfunclet$?sl_clipboardCheck@BrowserSupportPlugin@U2@@IAEXXZ$26 10004a45 f   BrowserSupportPlugin.obj
 0001:00003a5e       __unwindfunclet$?sl_clipboardCheck@BrowserSupportPlugin@U2@@IAEXXZ$27 10004a5e f   BrowserSupportPlugin.obj
 0001:00003a78       __unwindfunclet$?sl_clipboardCheck@BrowserSupportPlugin@U2@@IAEXXZ$28 10004a78 f   BrowserSupportPlugin.obj
 0001:00003a81       __unwindfunclet$?sl_clipboardCheck@BrowserSupportPlugin@U2@@IAEXXZ$29 10004a81 f   BrowserSupportPlugin.obj
 0001:00003a8a       __unwindfunclet$?sl_clipboardCheck@BrowserSupportPlugin@U2@@IAEXXZ$30 10004a8a f   BrowserSupportPlugin.obj
 0001:00003a98       __unwindfunclet$?sl_clipboardCheck@BrowserSupportPlugin@U2@@IAEXXZ$31 10004a98 f   BrowserSupportPlugin.obj
 0001:00003aa1       __unwindfunclet$?sl_clipboardCheck@BrowserSupportPlugin@U2@@IAEXXZ$32 10004aa1 f   BrowserSupportPlugin.obj
 0001:00003aaa       __unwindfunclet$?sl_clipboardCheck@BrowserSupportPlugin@U2@@IAEXXZ$33 10004aaa f   BrowserSupportPlugin.obj
 0001:00003ab3       __unwindfunclet$?sl_clipboardCheck@BrowserSupportPlugin@U2@@IAEXXZ$34 10004ab3 f   BrowserSupportPlugin.obj
 0001:00003abc       __unwindfunclet$?sl_clipboardCheck@BrowserSupportPlugin@U2@@IAEXXZ$35 10004abc f   BrowserSupportPlugin.obj
 0001:00003ac5       __unwindfunclet$?sl_clipboardCheck@BrowserSupportPlugin@U2@@IAEXXZ$36 10004ac5 f   BrowserSupportPlugin.obj
 0001:00003ace       __unwindfunclet$?sl_clipboardCheck@BrowserSupportPlugin@U2@@IAEXXZ$37 10004ace f   BrowserSupportPlugin.obj
 0001:00003ad9       __unwindfunclet$?sl_clipboardCheck@BrowserSupportPlugin@U2@@IAEXXZ$38 10004ad9 f   BrowserSupportPlugin.obj
 0001:00003af3       __unwindfunclet$?sl_clipboardCheck@BrowserSupportPlugin@U2@@IAEXXZ$39 10004af3 f   BrowserSupportPlugin.obj
 0001:00003b0c       __unwindfunclet$?sl_clipboardCheck@BrowserSupportPlugin@U2@@IAEXXZ$40 10004b0c f   BrowserSupportPlugin.obj
 0001:00003b26       __unwindfunclet$?sl_clipboardCheck@BrowserSupportPlugin@U2@@IAEXXZ$41 10004b26 f   BrowserSupportPlugin.obj
 0001:00003b2f       __ehhandler$?sl_clipboardCheck@BrowserSupportPlugin@U2@@IAEXXZ 10004b2f f   BrowserSupportPlugin.obj
 0001:00003b50       ??__F?_Generic_object@?$_Error_objects@H@std@@2V_Generic_error_category@2@A@@YAXXZ 10004b50 f   BrowserSupportPlugin.obj
 0001:00003b60       ??__F?_Iostream_object@?$_Error_objects@H@std@@2V_Iostream_error_category@2@A@@YAXXZ 10004b60 f   BrowserSupportPlugin.obj
 0001:00003b70       ??__F?_System_object@?$_Error_objects@H@std@@2V_System_error_category@2@A@@YAXXZ 10004b70 f   BrowserSupportPlugin.obj
 0001:00003b80       ??__FalgoLog@U2@@YAXXZ     10004b80 f   BrowserSupportPlugin.obj
 0001:00003b90       ??__FcmdLog@U2@@YAXXZ      10004b90 f   BrowserSupportPlugin.obj
 0001:00003ba0       ??__FcoreLog@U2@@YAXXZ     10004ba0 f   BrowserSupportPlugin.obj
 0001:00003bb0       ??__Fcvar@?BB@??sl_clipboardCheck@BrowserSupportPlugin@U2@@IAEXXZ@YAXXZ 10004bb0 f   BrowserSupportPlugin.obj
 0001:00003bc0       ??__Fcvar@?BE@??sl_clipboardCheck@BrowserSupportPlugin@U2@@IAEXXZ@YAXXZ 10004bc0 f   BrowserSupportPlugin.obj
 0001:00003bd0       ??__Fcvar@?L@??sl_clipboardCheck@BrowserSupportPlugin@U2@@IAEXXZ@YAXXZ 10004bd0 f   BrowserSupportPlugin.obj
 0001:00003be0       ??__FioLog@U2@@YAXXZ       10004be0 f   BrowserSupportPlugin.obj
 0001:00003bf0       ??__FperfLog@U2@@YAXXZ     10004bf0 f   BrowserSupportPlugin.obj
 0001:00003c00       ??__FprevClipboard@U2@@YAXXZ 10004c00 f   BrowserSupportPlugin.obj
 0001:00003c10       ??__FscriptLog@U2@@YAXXZ   10004c10 f   BrowserSupportPlugin.obj
 0001:00003c20       ??__FtaskLog@U2@@YAXXZ     10004c20 f   BrowserSupportPlugin.obj
 0001:00003c30       ??__FuiLog@U2@@YAXXZ       10004c30 f   BrowserSupportPlugin.obj
 0001:00003c40       ??__FuserActLog@U2@@YAXXZ  10004c40 f   BrowserSupportPlugin.obj
 0001:00003c50       ??__F?_Generic_object@?$_Error_objects@H@std@@2V_Generic_error_category@2@A@@YAXXZ 10004c50 f   moc_BrowserSupportPlugin.obj
 0001:00003c60       ??__F?_Iostream_object@?$_Error_objects@H@std@@2V_Iostream_error_category@2@A@@YAXXZ 10004c60 f   moc_BrowserSupportPlugin.obj
 0001:00003c70       ??__F?_System_object@?$_Error_objects@H@std@@2V_System_error_category@2@A@@YAXXZ 10004c70 f   moc_BrowserSupportPlugin.obj
 0002:0000023c       _algoLog$initializer$      1000523c     BrowserSupportPlugin.obj
 0002:00000240       _cmdLog$initializer$       10005240     BrowserSupportPlugin.obj
 0002:00000244       _coreLog$initializer$      10005244     BrowserSupportPlugin.obj
 0002:00000248       _ioLog$initializer$        10005248     BrowserSupportPlugin.obj
 0002:0000024c       _perfLog$initializer$      1000524c     BrowserSupportPlugin.obj
 0002:00000250       _scriptLog$initializer$    10005250     BrowserSupportPlugin.obj
 0002:00000254       _taskLog$initializer$      10005254     BrowserSupportPlugin.obj
 0002:00000258       _uiLog$initializer$        10005258     BrowserSupportPlugin.obj
 0002:0000025c       _userActLog$initializer$   1000525c     BrowserSupportPlugin.obj
 0002:00000260       _prevClipboard$initializer$ 10005260     BrowserSupportPlugin.obj
 0002:00000264       ?_Generic_object$initializer$@?$_Error_objects@H@std@@2P6AXXZA 10005264     BrowserSupportPlugin.obj
 0002:00000268       ?_Iostream_object$initializer$@?$_Error_objects@H@std@@2P6AXXZA 10005268     BrowserSupportPlugin.obj
 0002:0000026c       ?_System_object$initializer$@?$_Error_objects@H@std@@2P6AXXZA 1000526c     BrowserSupportPlugin.obj
 0002:00000270       ?staticMetaObject$initializer$@BrowserSupportPlugin@U2@@2P6AXXZA 10005270     moc_BrowserSupportPlugin.obj
 0002:0000027c       _pcinit                    1000527c     MSVCRT:crtdll.obj
 0002:00000280       _pinit                     10005280     MSVCRT:atonexit.obj
 0002:000005e0       _qt_meta_stringdata_U2__BrowserSupportPlugin 100055e0     moc_BrowserSupportPlugin.obj
 0002:00000640       _qt_meta_data_U2__BrowserSupportPlugin 10005640     moc_BrowserSupportPlugin.obj
 0002:000006a4       _GS_ExceptionPointers      100056a4     MSVCRT:gs_report.obj
 0002:00000a98       __catchsym$?_Copy@?$basic_string@DU?$char_traits@D@std@@V?$allocator@D@2@@std@@QAEXII@Z$5 10005a98     BrowserSupportPlugin.obj
 0002:00000aa8       __catchsym$?_Copy@?$basic_string@DU?$char_traits@D@std@@V?$allocator@D@2@@std@@QAEXII@Z$4 10005aa8     BrowserSupportPlugin.obj
 0002:00000ab8       __unwindtable$?_Copy@?$basic_string@DU?$char_traits@D@std@@V?$allocator@D@2@@std@@QAEXII@Z 10005ab8     BrowserSupportPlugin.obj
 0002:00000ad8       __ehfuncinfo$?_Copy@?$basic_string@DU?$char_traits@D@std@@V?$allocator@D@2@@std@@QAEXII@Z 10005ad8     BrowserSupportPlugin.obj
 0002:00000afc       __tryblocktable$?_Copy@?$basic_string@DU?$char_traits@D@std@@V?$allocator@D@2@@std@@QAEXII@Z 10005afc     BrowserSupportPlugin.obj
 0002:00000b24       __unwindtable$??__EalgoLog@U2@@YAXXZ 10005b24     BrowserSupportPlugin.obj
 0002:00000b2c       __ehfuncinfo$??__EalgoLog@U2@@YAXXZ 10005b2c     BrowserSupportPlugin.obj
 0002:00000b50       __unwindtable$??__EcmdLog@U2@@YAXXZ 10005b50     BrowserSupportPlugin.obj
 0002:00000b58       __ehfuncinfo$??__EcmdLog@U2@@YAXXZ 10005b58     BrowserSupportPlugin.obj
 0002:00000b7c       __unwindtable$??__EcoreLog@U2@@YAXXZ 10005b7c     BrowserSupportPlugin.obj
 0002:00000b84       __ehfuncinfo$??__EcoreLog@U2@@YAXXZ 10005b84     BrowserSupportPlugin.obj
 0002:00000ba8       __unwindtable$??__EioLog@U2@@YAXXZ 10005ba8     BrowserSupportPlugin.obj
 0002:00000bb0       __ehfuncinfo$??__EioLog@U2@@YAXXZ 10005bb0     BrowserSupportPlugin.obj
 0002:00000bd4       __unwindtable$??__EperfLog@U2@@YAXXZ 10005bd4     BrowserSupportPlugin.obj
 0002:00000bdc       __ehfuncinfo$??__EperfLog@U2@@YAXXZ 10005bdc     BrowserSupportPlugin.obj
 0002:00000c00       __unwindtable$??__EscriptLog@U2@@YAXXZ 10005c00     BrowserSupportPlugin.obj
 0002:00000c08       __ehfuncinfo$??__EscriptLog@U2@@YAXXZ 10005c08     BrowserSupportPlugin.obj
 0002:00000c2c       __unwindtable$??__EtaskLog@U2@@YAXXZ 10005c2c     BrowserSupportPlugin.obj
 0002:00000c34       __ehfuncinfo$??__EtaskLog@U2@@YAXXZ 10005c34     BrowserSupportPlugin.obj
 0002:00000c58       __unwindtable$??__EuiLog@U2@@YAXXZ 10005c58     BrowserSupportPlugin.obj
 0002:00000c60       __ehfuncinfo$??__EuiLog@U2@@YAXXZ 10005c60     BrowserSupportPlugin.obj
 0002:00000c84       __unwindtable$??__EuserActLog@U2@@YAXXZ 10005c84     BrowserSupportPlugin.obj
 0002:00000c8c       __ehfuncinfo$??__EuserActLog@U2@@YAXXZ 10005c8c     BrowserSupportPlugin.obj
 0002:00000cb0       __catchsym$?append@?$QList@VGUrl@U2@@@@QAEXABVGUrl@U2@@@Z$11 10005cb0     BrowserSupportPlugin.obj
 0002:00000cc0       __catchsym$?append@?$QList@VGUrl@U2@@@@QAEXABVGUrl@U2@@@Z$10 10005cc0     BrowserSupportPlugin.obj
 0002:00000cd0       __ehfuncinfo$?append@?$QList@VGUrl@U2@@@@QAEXABVGUrl@U2@@@Z 10005cd0     BrowserSupportPlugin.obj
 0002:00000cf4       __tryblocktable$?append@?$QList@VGUrl@U2@@@@QAEXABVGUrl@U2@@@Z 10005cf4     BrowserSupportPlugin.obj
 0002:00000d1c       __unwindtable$?append@?$QList@VGUrl@U2@@@@QAEXABVGUrl@U2@@@Z 10005d1c     BrowserSupportPlugin.obj
 0002:00000d6c       __catchsym$?detach_helper_grow@?$QList@VGUrl@U2@@@@AAEPAUNode@1@HH@Z$5 10005d6c     BrowserSupportPlugin.obj
 0002:00000d7c       __catchsym$?detach_helper_grow@?$QList@VGUrl@U2@@@@AAEPAUNode@1@HH@Z$4 10005d7c     BrowserSupportPlugin.obj
 0002:00000d8c       __unwindtable$?detach_helper_grow@?$QList@VGUrl@U2@@@@AAEPAUNode@1@HH@Z 10005d8c     BrowserSupportPlugin.obj
 0002:00000dac       __ehfuncinfo$?detach_helper_grow@?$QList@VGUrl@U2@@@@AAEPAUNode@1@HH@Z 10005dac     BrowserSupportPlugin.obj
 0002:00000dd0       __tryblocktable$?detach_helper_grow@?$QList@VGUrl@U2@@@@AAEPAUNode@1@HH@Z 10005dd0     BrowserSupportPlugin.obj
 0002:00000df8       __unwindtable$?node_construct@?$QList@VGUrl@U2@@@@AAEXPAUNode@1@ABVGUrl@U2@@@Z 10005df8     BrowserSupportPlugin.obj
 0002:00000e08       __ehfuncinfo$?node_construct@?$QList@VGUrl@U2@@@@AAEXPAUNode@1@ABVGUrl@U2@@@Z 10005e08     BrowserSupportPlugin.obj
 0002:00000e2c       __catchsym$?node_copy@?$QList@VGUrl@U2@@@@AAEXPAUNode@1@00@Z$6 10005e2c     BrowserSupportPlugin.obj
 0002:00000e3c       __tryblocktable$?node_copy@?$QList@VGUrl@U2@@@@AAEXPAUNode@1@00@Z 10005e3c     BrowserSupportPlugin.obj
 0002:00000e50       __ehfuncinfo$?node_copy@?$QList@VGUrl@U2@@@@AAEXPAUNode@1@00@Z 10005e50     BrowserSupportPlugin.obj
 0002:00000e74       __unwindtable$?node_copy@?$QList@VGUrl@U2@@@@AAEXPAUNode@1@00@Z 10005e74     BrowserSupportPlugin.obj
 0002:00000ea4       __ehfuncinfo$??0BrowserSupportPlugin@U2@@QAE@XZ 10005ea4     BrowserSupportPlugin.obj
 0002:00000ec8       __unwindtable$??0BrowserSupportPlugin@U2@@QAE@XZ 10005ec8     BrowserSupportPlugin.obj
 0002:00000ef0       __ehfuncinfo$?sl_clipboardCheck@BrowserSupportPlugin@U2@@IAEXXZ 10005ef0     BrowserSupportPlugin.obj
 0002:00000f14       __unwindtable$?sl_clipboardCheck@BrowserSupportPlugin@U2@@IAEXXZ 10005f14     BrowserSupportPlugin.obj
 0002:0000109c       __ehfuncinfo$?saveToTmp@BrowserSupportPlugin@U2@@IAE?AVQString@@AAV3@@Z 1000609c     BrowserSupportPlugin.obj
 0002:000010c0       __unwindtable$?saveToTmp@BrowserSupportPlugin@U2@@IAE?AVQString@@AAV3@@Z 100060c0     BrowserSupportPlugin.obj
 0002:00001108       __sehtable$__onexit        10006108     MSVCRT:atonexit.obj
 0002:00001128       __sehtable$___DllMainCRTStartup 10006128     MSVCRT:crtdll.obj
 0002:00001150       __sehtable$??_M@YGXPAXIHP6EX0@Z@Z 10006150     MSVCRT:ehvecdtr.obj
 0002:00001170       __sehtable$?__ArrayUnwind@@YGXPAXIHP6EX0@Z@Z 10006170     MSVCRT:ehvecdtr.obj
 0002:00001190       __sehtable$__IsNonwritableInCurrentImage 10006190     MSVCRT:pesect.obj
 0002:000011b0       .edata                     100061b0     browser_support.exp
 0002:000011d8       rgpv                       100061d8     browser_support.exp
 0002:000011dc       rgszName                   100061dc     browser_support.exp
 0002:000011e0       rgwOrd                     100061e0     browser_support.exp
 0002:000011e2       szName                     100061e2     browser_support.exp
 0002:000011f6       $N00001                    100061f6     browser_support.exp
 0002:00001cac       .idata$6                   10006cac     U2Core:U2Core.dll
 0002:00001f50       .idata$6                   10006f50     U2Gui:U2Gui.dll
 0002:00001ff0       .idata$6                   10006ff0     Qt5Gui:Qt5Gui.dll
 0002:0000262c       .idata$6                   1000762c     Qt5Core:Qt5Core.dll
 0002:000026d2       .idata$6                   100076d2     msvcprt:MSVCP120.dll
 0002:00002756       .idata$6                   10007756     MSVCRT:MSVCR120.dll
 0002:0000296a       .idata$6                   1000796a     kernel32:KERNEL32.dll
 0003:000001a0       __Tuple_alloc              100081a0     BrowserSupportPlugin.obj
 0003:000001a1       _ignore                    100081a1     BrowserSupportPlugin.obj
 0003:000001a2       _allocator_arg             100081a2     BrowserSupportPlugin.obj
 0003:000001a3       _piecewise_construct       100081a3     BrowserSupportPlugin.obj
 0003:000001a4       _taskLog                   100081a4     BrowserSupportPlugin.obj
 0003:000001ac       _algoLog                   100081ac     BrowserSupportPlugin.obj
 0003:000001b4       _userActLog                100081b4     BrowserSupportPlugin.obj
 0003:000001bc       _ioLog                     100081bc     BrowserSupportPlugin.obj
 0003:000001c4       _coreLog                   100081c4     BrowserSupportPlugin.obj
 0003:000001cc       _prevClipboard             100081cc     BrowserSupportPlugin.obj
 0003:000001d0       _uiLog                     100081d0     BrowserSupportPlugin.obj
 0003:000001d8       _scriptLog                 100081d8     BrowserSupportPlugin.obj
 0003:000001e0       _perfLog                   100081e0     BrowserSupportPlugin.obj
 0003:000001e8       _cmdLog                    100081e8     BrowserSupportPlugin.obj
 0003:000001f8       ?cvar@?L@??sl_clipboardCheck@BrowserSupportPlugin@U2@@IAEXXZ@4VGReportableCounter@3@A 100081f8     BrowserSupportPlugin.obj
 0003:00000220       ?$S1@?L@??sl_clipboardCheck@BrowserSupportPlugin@U2@@IAEXXZ@4IA 10008220     BrowserSupportPlugin.obj
 0003:00000228       ?cvar@?BB@??sl_clipboardCheck@BrowserSupportPlugin@U2@@IAEXXZ@4VGReportableCounter@3@A 10008228     BrowserSupportPlugin.obj
 0003:00000250       ?cvar@?BE@??sl_clipboardCheck@BrowserSupportPlugin@U2@@IAEXXZ@4VGReportableCounter@3@A 10008250     BrowserSupportPlugin.obj
 0003:00000278       __Tuple_alloc              10008278     moc_BrowserSupportPlugin.obj
 0003:00000279       _ignore                    10008279     moc_BrowserSupportPlugin.obj
 0003:0000027a       _allocator_arg             1000827a     moc_BrowserSupportPlugin.obj
 0003:0000027b       _piecewise_construct       1000827b     moc_BrowserSupportPlugin.obj
 0003:0000027c       ___proc_attached           1000827c     MSVCRT:crtdll.obj
 0003:00000280       _GS_ExceptionRecord        10008280     MSVCRT:gs_report.obj
 0003:000002d0       _GS_ContextRecord          100082d0     MSVCRT:gs_report.obj
 0003:0000059c       _DebuggerWasPresent        1000859c     MSVCRT:gs_report.obj
 0004:00000060       $R000000                   10009060     * linker generated manifest res *

 Exports

  ordinal    name

        1    _ugene_plugin_init
               exported name: ugene_plugin_init
